:100000000C94C8000C940E370C943A0E0C94E50036
:100010000C94E5000C94E5000C94E5000C94E500CC
:100020000C94E5000C94E5000C94E5000C94A810E9
:100030000C94E5000C94502F0C948A2F0C94B32F41
:100040000C94E5000C94E5000C94E5000C944F38FA
:100050000C94E50031313056332E33350000000169
:100060000000060000FF00000F02000C0014010158
:100070000400001450040100000000000000000013
:1000800000000000010003E8000000000000000381
:10009000E800000000000200FA0600070000FF0070
:1000A0000037060002800000000000002107101049
:1000B0000504030206100D0C0B0A2E1005040302A2
:1000C00006100D0C0B0A2E100504030206100D0C71
:1000D0000B0A2E1111111111111111111111111100
:1000E0001111111111111111111111111111110011
:1000F0000404040808080C0C0C1010101414181830
:10010000181C1C1C20202020242424282828282CCB
:100110002C2C2C30303030343434343438383838B7
:10012000383838383C3C3C3C3C3C3C3C3C3C3C1843
:10013000180B0B0C0C0B0C0B040208040C1803031B
:10014000030801010101010804040101000000008D
:1001500000000C10140808090A0B0C08080C090A06
:100160000B0C0D0E080808090A0A0A0A0A0B0C0CE7
:1001700000010405030647401D1B1C1B14133322FA
:1001800019100C080603016744332219100C0803E8
:1001900011241FBECFE5D8E0DEBFCDBF11E0A0E641
:1001A000B0E0E6E4F6E702C005900D92A031B10799
:1001B000D9F716E0A0E1B1E001C01D92A137B10767
:1001C000E1F70E94E7000C94223B0C940000AF92F0
:1001D000BF92CF92DF92EF92FF920F931F93CF9334
:1001E000DF93CDB7DEB724970FB6F894DEBF0FBE0E
:1001F000CDBF0E94FD0E82E00E9481100E94770F09
:100200008DB18F738DB981E887BB30E020E018BADB
:1002100000000000000096B380E888BB00000000EA
:100220000000B69B02C096FF2F5F3F5F3A3079F720
:100230002A3039F560E089E090E00E94EE0F60E03E
:1002400080E090E00E94EE0F1A82198205C0898139
:100250009A8101969A83898389819A818F5F9F4FC2
:10026000B1F7C0981A82198205C089819A810196D6
:100270009A83898389819A818F5F9F4FB1F7C09A52
:10028000E3CF0E94FD0E82E00E9481100E944C0E7E
:100290000E9403110E94770FAB980E943E0F0E94AC
:1002A000540F80E090E00E94E60F843E09F4F9C00C
:1002B000C0980E946F3060E089E090E00E94EE0FED
:1002C00040E16DE570E080E090E00E94331061E075
:1002D0008AE491E00E94EE0F60E08BE491E00E94DE
:1002E000EE0F60E08CE491E00E94EE0F60E08DE4A0
:1002F00091E00E94EE0F62E08EE491E00E94EE0F2A
:1003000060E08FE491E00E94EE0F60E080E591E014
:100310000E94EE0F60E081E591E00E94EE0F60E048
:1003200085E192E00E94EE0F60E086E192E00E949B
:10033000EE0F60E087E192E00E94EE0F60E088E15E
:1003400092E00E94EE0F0E940B104DE26CE770E00D
:100350008DE390E00E9433104DE26CE770E08AE696
:1003600090E00E9433104DE26CE770E087E990E086
:100370000E94331043E069EA70E084EC90E00E9450
:10038000331043E06CEA70E087EC90E00E94331099
:1003900040E86FEA70E08AEC90E00E94331064E677
:1003A0008AE591E00E94EE0F60E08BE591E00E940B
:1003B000EE0F64E68CE591E00E94EE0F60E08DE5C3
:1003C00091E00E94EE0F64E68EE591E00E94EE0F50
:1003D00060E08FE591E00E94EE0F60E080E691E042
:1003E0000E94EE0F60E081E691E00E94EE0F60E077
:1003F00082E691E00E94EE0F60E083E691E00E94C9
:10040000EE0F60E084E691E00E94EE0F60E085E68A
:1004100091E00E94EE0F60E08DEF93E00E94EE0FFE
:1004200060E08EEF93E00E94EE0F60E08FEF93E0CC
:100430000E94EE0F60E086E691E00E94EE0F68E019
:1004400087E691E00E94EE0F60E088E691E00E946E
:10045000EE0F68E089E691E00E94EE0F60E08AE628
:1004600091E00E94EE0F68E08BE691E00E94EE0FB3
:1004700060E089E192E00E94EE0F60E08AE192E0A4
:100480000E94EE0F81E090E00E94E60FEEE5F0E0C2
:10049000E4918E1729F464EE80E090E00E94EE0F64
:1004A000C09A81E090E00E94E60F0E94C82F8AE087
:1004B00090E00E94E60F8093BD04882311F00E9413
:1004C00053398EE70E941D0B10E0812F80610E943E
:1004D0001D0B812F88610E941D0B812F84600E945B
:1004E0001D0B812F86600E941D0B812F84610E944D
:1004F0001D0B105E103649F70E949C090E945B108C
:10050000EE24FF24C70125E0880F991F2A95E1F703
:100510008D600E94B80F082F10E0C80101960E945C
:10052000E60F8C83C80102960E94E60F8B836B81D5
:100530007C818E2D0E945808C70185960E94E60F87
:10054000682F8E2D0E94B50F0894E11CF11C83E0EA
:10055000E816F104B9F62FEF4FEF60E086E10E9454
:10056000A0052FEF4FEF60E086E30E94A0052FEF7C
:100570004FEF60E086E50E94A0058AE491E00E94CA
:10058000E60F809330068BE491E00E94E60F8093A3
:1005900031068CE491E00E94E60F809332068DE4F0
:1005A00091E00E94E60F809333068EE491E00E9472
:1005B000E60F8093E8058FE491E00E94E60F8093B8
:1005C000E90580E591E00E94E60F8093EA0581E568
:1005D00091E00E94E60F8093EB0585E192E00E9496
:1005E000E60F8093DC0586E192E00E94E60F80939F
:1005F000DD0587E192E00E94E60F8093DE0588E149
:1006000092E00E94E60F8093DF05E090DC05F09019
:10061000DD050091DE051091DF05A0903006B09059
:100620003106C0903206D090330685E090E00E94FB
:10063000E60F98018701B601A50190E00E94BA3447
:100640008AE591E00E94E60F809311068BE591E028
:100650000E94E60F809312068CE591E00E94E60F5F
:10066000809313068DE591E00E94E60F80931406B7
:100670008EE591E00E94E60F809315068FE591E0EC
:100680000E94E60F8093160680E691E00E94E60F36
:100690008093F30581E691E00E94E60F8093F405D4
:1006A00082E691E00E94E60F8093F50583E691E0F3
:1006B0000E94E60F8093F60584E691E00E94E60F23
:1006C0008093F70585E691E00E94E60F8093F80598
:1006D0008DEF93E00E94E60F809318068EEF93E073
:1006E0000E94E60F809319068FEF93E00E94E60FB9
:1006F00080931A0686E691E00E94E60F80935701E8
:1007000087E691E00E94E60F8093580188E691E029
:100710000E94E60F8093590189E691E00E94E60F5E
:1007200080935A018AE691E00E94E60F80935B0174
:100730008BE691E00E94E60F80935C0182E090E0FE
:100740000E94E60F0E9410380E94CF2E0E94D5030F
:10075000789489E192E00E94E60F8093D6058AE1C1
:1007600092E00E94E60F8093D7058091D605909184
:10077000D7058F5F9F4F21F41092D7051092D605B1
:100780008091D6059091D7059093D5058093D40597
:100790000E945B060E9409110E94530B0E9493293C
:1007A0000E94BF350E94DB03F3CF81E08093CB042E
:1007B0001092AC0508958091340681FF07C08091A6
:1007C000AC058F3F19F08F5F8093AC058091CB040F
:1007D000813051F48091AC058F3030F0C098109288
:1007E000AC0582E08093CB048091CB04823051F43D
:1007F0008091AC05853030F0C09A1092AC0581E054
:100800008093CB0408950895089508950895089558
:1008100008950895CF92DF92FF920F931F93CF9385
:10082000DF93CDB7DEB729970FB6F894DEBF0FBEC2
:10083000CDBF82E00E9430118CE090E00E94E60F74
:10084000898382E090E00E94E60F8A8381E88B83AF
:1008500081E48C838091C5058D838091C4058E834E
:100860008091C6058F838091C805888719868E017F
:100870000F5F1F4F89E0C82ED12CCC0EDD1EF80172
:10088000F0808985F80EF98680915E01882319F43D
:1008900080810E9414300F5F1F4F0C151D0579F7E2
:1008A00080915E01882319F48F2D0E9414302996BF
:1008B0000FB6F894DEBF0FBECDBFDF91CF911F9171
:1008C0000F91FF90DF90CF900895682F70E080FD2A
:1008D0002FC0CB018076907035E0959587953A953D
:1008E000E1F7E82FCB018F7990708431910529F4DD
:1008F000F0E0E35DF94F208308958630910541F4DF
:10090000F0E0EE0FFF1FE253FA4F2083418308957A
:10091000089771F4F0E0EE0FFF1FE95DF94F2083B7
:10092000418343FF05C080819181906F91838083D3
:100930000895EF92FF920F931F93182F062FF42E16
:10094000E22E0E9465048BB78F7B8BBFC398812FEB
:100950000E949010802F0E9490108F2D0E94901066
:100960008E2D0E949010C39A8BB780648BBF1F910D
:100970000F91FF90EF900895CF92DF92EF92FF9248
:100980000F931F93CF93DF937C016B01FC01808158
:1009900090E09C012F7930702115310519F0283035
:1009A0003105E1F4EC01C076D07045E0D595C795EE
:1009B0004A95E1F7C33090F48C2F8B5E0E946D1046
:1009C000682F8C2F0E94B50FEC2FF0E0DF01A054B0
:1009D000BA4F83E08C93E550FA4F1082F7012381E0
:1009E0004281618180810E9465048BB78F7B8BBFC0
:1009F000C398C0E0D0E086010C0F1D1FF701EC0F7B
:100A0000FD1F80810E949010F80180832196C430E0
:100A1000D10589F7C39A8BB780648BBF80E090E0E3
:100A2000DF91CF911F910F91FF90EF90DF90CF90CA
:100A300008955F926F927F928F929F92AF92BF9232
:100A4000CF92DF92EF92FF920F931F93CF93DF939A
:100A5000CDB7DEB728970FB6F894DEBF0FBECDBF77
:100A60001A829CE0899FC0011124B0E85B2E580EC9
:100A700000E010E070E0A4E0AA2EB12CA622B7227C
:100A8000F2E0CF2ED12CC622D722E1E0EE2EF12CBF
:100A9000E622F72255E0652E712C6C0E7D1E4E016C
:100AA0000894811C911CA114B10489F0063020F433
:100AB000E114F10421F006C0C114D10419F490E14D
:100AC00080E102C091E181E18B839C830CC0C8016D
:100AD00085539F4F0E94E60F8B83C80186539F4F1B
:100AE0000E94E60F8C83902F002311F0063011F442
:100AF00080E18C839A3019F48B8180628B83950D11
:100B00009983B301C4010E94BC040E5F1F4F0C30D7
:100B1000110549F628960FB6F894DEBF0FBECDBF7B
:100B2000DF91CF911F910F91FF90EF90DF90CF90C9
:100B3000BF90AF909F908F907F906F905F9008953F
:100B40003F924F925F926F927F928F929F92AF925D
:100B5000BF92CF92DF92EF92FF920F931F93CF93AA
:100B6000DF93CDB7DEB728970FB6F894DEBF0FBE80
:100B7000CDBFC82E562E442E322E90E09C012F79E8
:100B800030702115310521F02830310509F061C0A0
:100B90008076907045E0959587954A95E1F7D82E37
:100BA00082E08D1508F455C0ED2CFF24F701EE0FFF
:100BB000FF1FDF01AD50BA4F8D919C91E25BFE4F5C
:100BC00091838083F701EC5AFE4F8081882371F175
:100BD00010821A828CE0D89EC00111248C0100582A
:100BE0001F4F2CE8A22EB12CA80EB91E85E0682E4E
:100BF000712C6C0E7D1E4E010894811C911C13C03B
:100C00000983C801855B9F4F0E94E60F8B83C80153
:100C1000865B9F4F0E94E60F8C83B301C4010E9444
:100C2000BC040E5F1F4F0A151B0550F38D2D8B5E04
:100C30000E946D10682F8D2D0E94B50FF701E054B2
:100C4000FA4F83E08083EBEFF5E0EE0EFF1EF70135
:100C50001082232D442D652D8C2D0E9465048BB7A9
:100C60008F7B8BBFC3988C2D0E949010852D0E9486
:100C70009010842D0E949010832D0E949010C39A92
:100C80008BB780648BBF28960FB6F894DEBF0FBE7B
:100C9000CDBFDF91CF911F910F91FF90EF90DF902B
:100CA000CF90BF90AF909F908F907F906F905F900C
:100CB0004F903F900895AF92BF92CF92DF92EF9204
:100CC000FF920F931F93CF93DF93CDB7DEB72A9791
:100CD0000FB6F894DEBF0FBECDBF1092B5051092CF
:100CE000B6051092B7058091BE05882311F083994F
:100CF0005FC0809110018F5F80931001833010F0EE
:100D0000109210018EE090E00E94E60F8F5F8093BA
:100D1000BE05809110018295880F807E8B608F8345
:100D20008E010D5F1F4F67E0C62ED12CCC0EDD1E4D
:100D3000B801C6010E94BC048B818093BF058D81E0
:100D400083FF02C0806F8D838D818A838E8189832A
:100D5000E0911001F0E0EE0FFF1FE854FA4F898197
:100D60009A8191838083839923C0EE24FF245801C4
:100D70001E2D1295110F107E812F87618F83B50173
:100D8000C6010E94BC04F701EB54FA4F8E818083A8
:100D900016611F838FEF89878A87B501C6010E947C
:100DA000BC040894E11CF11C83E0E816F10401F78F
:100DB0002A960FB6F894DEBF0FBECDBFDF91CF915C
:100DC0001F910F91FF90EF90DF90CF90BF90AF9069
:100DD0000895CF93DF93EC0182E090E00E94E60F4C
:100DE0008093240190912101992359F08091340638
:100DF00080FF03C091509093210180912001816078
:100E00000EC080912301882339F0809120018061F8
:100E10008093200110922301809120018E7F809386
:100E2000200180912301882309F058C081E191E0DD
:100E30000E94E933882309F451C0209114013091B4
:100E40001501409116015091170180913006909143
:100E50003106A0913206B0913306281739074A07A8
:100E60005B0789F08091DC059091DD05A091DE059E
:100E7000B091DF050097A105B10581F12817390769
:100E80004A075B0759F580911101873008F488C043
:100E90009E01295F3F4F809124018F83E8E1F1E0BB
:100EA000DE0180818D93E90188819191890F88838A
:100EB00081E0EF31F807A9F780911101873011F433
:100EC00081E001C082E08093E0058091D605909199
:100ED000D7059093D5058093D4056DC080912301EB
:100EE000882379F468E0CE010E941C38882349F0F9
:100EF0008F8190912401890F8F8381E08093170661
:100F00005AC00E94F02F8F3F31F480912001806100
:100F1000809320013AC085E291E00E943030813018
:100F2000A1F584E18093210120912301222329F45A
:100F3000809125018093220125C09091220180910A
:100F400024019817D1F430912001932F946090934D
:100F5000200191FD12C0C20FD11D21978091250162
:100F60008883283051F494FF04C09F7E9093200121
:100F700006C036603093200102C0283018F010926D
:100F8000230103C02F5F209323011092E0051092EC
:100F900017068091200184FF06C08F7E8093200178
:100FA0008FEF9FEF0AC081FD03C080E090E005C095
:100FB0008D7F8093200181E090E0DF91CF910895B3
:100FC000FB0120813181280F391F35952795318309
:100FD0002083C9010895FF920F931F93F62E81601D
:100FE0008093D80501EE15E0B80188ED95E00E94E8
:100FF000BC040F0D111DF801808190E01F910F912D
:10100000FF90089581608093D80561EE75E088EDCA
:1010100095E00E94BC048091E40590E00895816011
:101020008093D80561EE75E088ED95E00E94BC04E0
:101030002091E30530E0522F44278091E40590E0B1
:10104000482B592B23FD02C0CA010895CA01906F95
:101050000895CF93DF93CDB7DEB724970FB6F894FA
:10106000DEBF0FBECDBF81608093D80561EE75E015
:1010700088ED95E00E94BC049091E20597FF03C0C3
:101080008FEF8C8301C01C829B838091E3058A8350
:101090008091E405898369817A818B819C81249682
:1010A0000FB6F894DEBF0FBECDBFDF91CF9108958C
:1010B000CF92DF92FF920F931F93CF93DF93CDB721
:1010C000DEB721970FB6F894DEBF0FBECDBF8B0100
:1010D000F82EF294FF0C70EEF7228F2D8961809329
:1010E000D80561EE75E088ED95E00E94BC04C8016A
:1010F0008070987F892B19F08FEF9FEF57C08091F8
:10110000E305982F9F709C5F82958F70981B0F3F0F
:101110001105F9F0F4F06801191694F0412F5527E4
:10112000202F60E08F2D8C600E94A00520E04FE70B
:1011300060E08F2D82610E94A00581E090E036C0C2
:10114000D594C79491508FEFC816D104E1F0DCF02C
:10115000E3CF68019D3094F0412F5527202F60E0A8
:101160008F2D8C600E94A0052DE040E060E08F2D67
:1011700082610E94A00582E090E018C0CC0CDD1CCA
:101180009F5FC7FEE7CF412F5527202F60E08F2DAF
:101190008C6099830E94A0059981292F4C2D60E0D5
:1011A0008F2D82610E94A00580E090E021960FB60D
:1011B000F894DEBF0FBECDBFDF91CF911F910F918D
:1011C000FF90DF90CF9008950F931F93062F182F55
:1011D0001295110F107E812F85618093D80561EEE5
:1011E00075E088ED95E00E94BC04202F4091E30556
:1011F00060E0812F84610E94A0051F910F910895E6
:10120000CF93DF93CDB7DEB724970FB6F894DEBF48
:101210000FBECDBF49835A836B837C8329814A816A
:101220006B810E94A00524960FB6F894DEBF0FBE16
:10123000CDBFDF91CF9108951F93182F62E00E94D8
:10124000E4081295110F107E40E050E060E070E07D
:10125000812F88600E94000940E050E060E070E06B
:10126000812F8A600E9400091F9108958295880F3E
:10127000807E40E050E060E070E088600E940009FD
:101280000895E82FF0E0EE0FFF1FE25AF94F40817A
:101290005181662329F002C0559547956A95E2F77A
:1012A000509541955F4F662757FD6095762F829543
:1012B000880F807E88600E9400090895E82FF0E082
:1012C000EE0FFF1FE25AF94F40815181662329F04A
:1012D00002C0559547956A95E2F7662757FD6095D8
:1012E000762F8295880F807E88600E94000908957D
:1012F0000F931F93CF93DF93CDB7DEB722970FB62F
:10130000F894DEBF0FBECDBF8C0101970E94E60F9F
:10131000FE0131968183C8010E94E60F898389818D
:101320009A8122960FB6F894DEBF0FBECDBFDF9133
:10133000CF911F910F910895CF92DF92EF92FF927C
:101340000F931F93CF93DF93CDB7DEB728970FB6D8
:10135000F894DEBF0FBECDBF1A820BEC10E085E023
:10136000C82ED12CCC0EDD1E7E010894E11CF11C90
:10137000802F8B548983C8010E94E60F8B83C8019C
:1013800001970E94E60F8C83B601C7010E94BC043E
:101390000E5F1F4F81E00B34180751F728960FB6E8
:1013A000F894DEBF0FBECDBFDF91CF911F910F919B
:1013B000FF90EF90DF90CF9008951F9390912C01B4
:1013C00080912B01981719F480E090E040C0E92F3C
:1013D000F0E0EF5BFE4F1081892F8F5F80932C012F
:1013E0008A3011F410922C01EEE1F6E0119286E0C1
:1013F000E732F807D9F78CE090E00E94E60F80937F
:101400001E0682E090E00E94E60F80931F0680E8AF
:10141000809320068AE88093210610932506209168
:101420001C06233019F4EFE1F6E005C080911E069A
:1014300080932606F8CF819190912606890F80939C
:10144000260686E0E632F807B1F7822F90E01F917A
:101450000895EF92FF920F931F938B01E82EFF24C4
:10146000C70125E0880F991F2A95E1F788610E943E
:101470000208877002C0000F111F8A95E2F7612FE2
:10148000772767FD7A95C7014C960E94EE0F602F73
:10149000C7014F960E94EE0F1F910F91FF90EF90A2
:1014A0000895CF92DF92EF92FF920F931F93CF9305
:1014B000DF93CDB7DEB728970FB6F894DEBF0FBE27
:1014C000CDBF1A820BE011E035E0C32ED12CCC0E3B
:1014D000DD1E7E010894E11CF11C802F8A54898353
:1014E000B601C7010E94BC046F81C8010E94EE0FC3
:1014F0006885C80101970E94EE0F0E5F1F4F81E0C3
:101500000B34180751F728960FB6F894DEBF0FBEBC
:10151000CDBFDF91CF911F910F91FF90EF90DF90A2
:10152000CF900895CF92DF92EF92FF920F931F9387
:10153000CF93DF93CDB7DEB728970FB6F894DEBF11
:101540000FBECDBF1A820BEC10E045E0C42ED12CAB
:10155000CC0EDD1E7E010894E11CF11C802F8A5404
:101560008983B601C7010E94BC046F81C8010E9433
:10157000EE0F6885C80101970E94EE0F0E5F1F4FA6
:1015800081E00B34180751F728960FB6F894DEBFA8
:101590000FBECDBFDF91CF911F910F91FF90EF90C4
:1015A000DF90CF9008950F931F93CF93DF93082F71
:1015B000816007FD24C08093D80561EE75E088ED59
:1015C00095E00E94BC04802F0E94B80FC1EED5E0C8
:1015D000002711270C1B1D0B080F111D6981C80165
:1015E0008C0F9D1F0E94EE0F823019F482E090E074
:1015F0001FC0219685E0C43ED80781F717C08093AD
:10160000D80561EE75E088ED95E00E94BC0410E01D
:101610006091E305C801855B9F4F0E94EE0F6091CA
:10162000E405C801865B9F4F0E94EE0F80E090E0CA
:10163000DF91CF911F910F910895FF920F931F9308
:10164000CF93DF93CDB7DEB728970FB6F894DEBF00
:101650000FBECDBFF82E0E94B80F082F10E0F98200
:10166000C8010E94E60F8A83C80101960E94E60F16
:101670008B83C80102960E94E60F8C83BE016B5FCC
:101680007F4FCE0101960E94BC0480E090E0289636
:101690000FB6F894DEBF0FBECDBFDF91CF911F9183
:1016A0000F91FF9008952F923F924F925F926F9209
:1016B0007F928F929F92AF92BF92CF92DF92EF92E2
:1016C000FF920F931F93CF93DF93CDB7DEB724978D
:1016D0000FB6F894DEBF0FBECDBF86E090E00E944B
:1016E000E60F8A8380913D018F5F80933D01815099
:1016F000823010F010923D0180912601882369F418
:1017000080E68093D80561EE75E088ED95E00E9453
:10171000BC041092270181E01BC08130E1F481E616
:101720008093D80561EE75E088ED95E00E94BC04D9
:101730008091E10586FD72C08091E30586958095D4
:1017400087708093E5058091E4058093FE0582E033
:101750008093260163C0823009F060C08091270128
:10176000A82FB0E0FD01E85EF94F9081992309F4BC
:1017700050C0FD01EB51FA4F8081891708F449C030
:1017800015E0AA0FBB1F1A95E1F78A2F8A600E9405
:101790000F08BC01892B09F43FC0A09127014A2FF3
:1017A00050E0FA01E35DF94F8081FA01EE0FFF1F6F
:1017B000882319F0E95DF94F02C0E253FA4F208106
:1017C0003181CB0177FF03C0909581959F4F37FF03
:1017D00003C0309521953F4F82179307E9F4FA0132
:1017E000E25CFE4F8081823078F08A2F0E941C09D3
:1017F000E0912701F0E0DF01A550BA4F81E08C9322
:10180000E25CFE4F108208C08F5F80831092260139
:1018100003C0A25CBE4F1C92109226018091340638
:1018200080FFAFC180E00E94A43181E00E94A4311A
:1018300082E00E94A4318DE78093D80561EE75E0C7
:1018400088ED95E00E94BC0410912C01E0912B01E1
:1018500070915D01A0E0B0E041E050E00A2E02C0CE
:10186000440F551F0A94E2F7642F842F8723D9F081
:101870008091E10590E09D01220F331F02C09595F4
:1018800087952A95E2F780FF0EC08E2F8F5F8A30F2
:1018900009F480E0811729F0F0E0EF5BFE4F408310
:1018A000E82F609576231196A330B105A9F6E09351
:1018B0002B0170935D018091340681FFAEC00BE473
:1018C00011E0E4E56E2EE1E07E2E78E2872E71E0F5
:1018D000972E61E1462E66E0562E50ECA52E55E07F
:1018E000B52E1C821B8240E8C42E36E8332EDB80E6
:1018F0008B819C8125E0880F991F2A95E1F78A60EA
:101900000E940F087C018091340682FF1EC0F50101
:101910008081E114F10461F0833041F08D2D8B5E04
:101920000E946D10682F8B810E94B50F83E00BC061
:10193000882341F48B810E946D10682F8B810E9457
:10194000B50F03C08150F5018083F2012081318100
:10195000FFEF2F3F3F07A9F4F8018081823009F49F
:1019600041C021E145E060E08C2D0E94990421E115
:101970004DE060E0832D0E94990482E0F8018083AD
:1019800031C0C701F7FE03C0909581959F4FF801C4
:1019900040818217930794F0413021F127E045E020
:1019A00060E08C2D0E9499042FE04DE060E0832DD3
:1019B0000E94990481E0F801808310C0442391F0D3
:1019C00020E145E060E08C2D0E94990420E14DE08B
:1019D00060E0832D0E949904F8011082F3011082C7
:1019E000F40110828B819C8101969C838B839CE007
:1019F000C90E390E0F5F1F4F0894611C711C0894AB
:101A0000811C911CE2E0F0E04E0E5F1E0894A11CC8
:101A1000B11CF4EACF1609F06ACF83EF282E85E0D7
:101A2000382E08E2C02E01E0D02E17E5412E11E03D
:101A3000512EB4E56B2EB1E07B2EAEE48A2EA1E0F0
:101A40009A2EAA24BB248AE88983C501F5E0880F71
:101A5000991FFA95E1F78A600E940F087C0197FFB1
:101A600004C0F094E194F108F394F1018081918134
:101A7000892B39F1E114F10421F5F4018081918180
:101A80000097D9F4F30180818823D9F419811A5081
:101A900000E020E140E160E0812F0E9499040E5FA8
:101AA0001E5F0C30B1F720E140E360E089810E94C5
:101AB000990481E0F301808304C00197F4019183CC
:101AC0008083AA2009F044C0F201808191810097AF
:101AD00009F4AFC0E816F90608F4ABC0F60180813E
:101AE000882309F0A6C081E0808300EC10E02CE29E
:101AF0004CE260E0802F0E9499040E5F1F4FF1E0DE
:101B000000301F0709F495C0F2CF892B09F5F601C3
:101B100080818823E9F01082EAE0EE2EE1E0FE2EDB
:101B2000C7010E94E60F182FC70101960E94E60F19
:101B3000212F482F60E08E2D8A540E94990482E064
:101B400090E0E80EF91E9AE4E91691E0F90641F7F3
:101B50000894A11CB11CE2E0F0E02E0E3F1E089498
:101B6000C11CD11C4E0E5F1EF981F45FF9830894ED
:101B7000611C711C82E090E0880E991EFE3A09F00B
:101B800064CF8091C3058823F9F484E08093C30572
:101B900068E081E096E00E94580FA7B1B0E0AA0F7C
:101BA000BB1FA35DBE4FE7B1F0E0EE0FFF1FEF5F7D
:101BB000F94F8D919C91119720813181820F931F54
:101BC000959587958D939C9390913D01E92FF0E039
:101BD000E051FA4F8081882319F0892F0E94B23199
:101BE0009A81992311F1EA81E13019F49A9906C09A
:101BF0001CC0FA81F230C9F49A9917C0AB9A81E0FF
:101C000080931B0600E010E062E0802F0E94E40851
:101C1000802F0E943609F801E051FA4F10820F5FC1
:101C20001F4F0330110569F0EFCFAB9810921B06E0
:101C300008C0F20180819181E816F90608F467CFA7
:101C400064CF24960FB6F894DEBF0FBECDBFDF91F0
:101C5000CF911F910F91FF90EF90DF90CF90BF90A9
:101C6000AF909F908F907F906F905F904F903F903C
:101C70002F9008951F920F920FB60F9211248F93F9
:101C800081E08093C7058F910F900FBE0F901F903A
:101C900018951092C70508951F93CF93DF93CDB782
:101CA000DEB722970FB6F894DEBF0FBECDBF23E09C
:101CB00040E060E084E10E94990423E040E060E0BD
:101CC00084E30E94990423E040E060E084E50E9400
:101CD000990420E040E060E08AE00E94990420E05E
:101CE00040E060E08AE20E94990420E040E060E089
:101CF0008AE40E94990410E002C01431A1F020E0AF
:101D000040E060E0812F0E94990420E040E060E024
:101D1000812F80620E94990420E040E060E0812FE2
:101D200080640E9499041E5F1C3138F320E040E07B
:101D300060E08EE70E94990410E020E040E060E05F
:101D4000812F80680E9499041E5F1038B1F72FEF31
:101D500047E060E08AE00E9499041A82198206C076
:101D6000000089819A8101969A83898389819A8169
:101D7000885B9B40ACF320E040E060E08AE00E949A
:101D800099048BB78F7B8BBFC39883E00E94901020
:101D900080E00E9490108093CB0580E00E9490101C
:101DA0008093CA0580E00E9490108093C905C39A71
:101DB0008BB780648BBF20E040E060E082E00E944F
:101DC00099048091C9059091CA05A091CB05B09165
:101DD000CC05805D9740A040B04010F480E101C088
:101DE00088E08093CD0522960FB6F894DEBF0FBE33
:101DF000CDBFDF91CF911F910895CF93DF93CDB7E2
:101E0000DEB722970FB6F894DEBF0FBECDBF8EEFC0
:101E10008ABB8CE08BBB8DEB87BB8FE188BB8CEFE3
:101E200084BB83EF85BB82EF81BB85E082BBDB98FF
:101E30001A82198206C0000089819A8101969A83CC
:101E4000898389819A8184369105ACF3DB9A1A8261
:101E5000198206C0000089819A8101969A8389833C
:101E600089819A8184369105ACF322960FB6F89455
:101E7000DEBF0FBECDBFDF91CF91089581B3806BE0
:101E800081BB81EF8FBD81E08EBD81E785BD089567
:101E9000882319F41BBC6ABD0895813019F419BC5C
:101EA00068BD089563BD089517B886EC86B9089596
:101EB00044B150E025B1E7B1F0E0EE0FFF1FE80FAD
:101EC000F91F30E0322F2227242B352B318320833A
:101ED00087B190E070E0615070408617970724F456
:101EE00087B18F5F87B901C017B8369A08950895F2
:101EF000882309F4D99A0895882309F4D998089574
:101F0000882319F080E090E0089589B390E0817013
:101F100090700895482F662359F02BB381E090E02C
:101F200002C0880F991F4A95E2F7282B2BBB089512
:101F30002BB381E090E002C0880F991F4A95E2F729
:101F4000809582238BBB0895882319F080E090E070
:101F500008958BB390E09695879581709070089561
:101F60008BBB089580E090E008950E94480F08958B
:101F7000282F87FD23C0482F46954F7083E0489F48
:101F8000C001112430E0207630702115310511F4A4
:101F9000CD961AC02032310519F486599F4F14C0CE
:101FA0002034310519F489569F4F0EC04F3019F473
:101FB00087EC90E009C04E3039F404C0265B822FD4
:101FC00090E0089583E090E090E00895DC01E199CD
:101FD000FECF0E94D73A802D90E008951F93CF93B3
:101FE000DF93EC01162F89E090E00E94E60F882332
:101FF00031F0C930D10519F082E090E008C0E199D4
:10200000FECFDE01012E0E94DF3A80E090E0DF91FA
:10201000CF911F910895EF92FF921F93CF93DF937B
:102020008DE6E82E80E0F82EC0E1D0E0F7011491B3
:10203000612FCE010E94EE0F612FCE0101960E940A
:10204000EE0F612FCE0102960E94EE0F0894E11C64
:10205000F11C2396CD33D10549F7DF91CF911F9124
:10206000FF90EF900895CF92DF92EF92FF920F933F
:102070001F93CF93DF936C017B01042F10E0C0E02E
:10208000D0E00CC0FE01EE0DFF1DE4916E2FCE01DD
:102090008C0D9D1D0E94EE0F1F5F2196101791F76A
:1020A00080E090E0DF91CF911F910F91FF90EF9032
:1020B000DF90CF900895CF93DF93C0E1D0E0CE01C1
:1020C0000E94E60FFE01E05BFE4F80832196CD3338
:1020D000D105A9F7DF91CF910895E0E6F1E0E80F8F
:1020E000F11D808190E008958D3218F081E090E03C
:1020F0000895E82FF0E0E05AFE4F608380E090E022
:10210000089583708DB98DB18C658DB9709A1092D8
:102110008D01089580918D0110928D0190E00895B8
:102120008FB980E009C0893C31F480918D018160D4
:1021300080938D0103C08F5F779BF5CF769B05C0A1
:1021400080918D01826080938D018FB190E0089520
:102150001F920F920FB60F9211248F939F93AF93FC
:10216000BF938091CD05883011F482E701C083E2EE
:1021700082BF80913506882319F0815080933506FF
:102180008091BE05882319F081508093BE0580910F
:102190009101882321F08150809391012BC088E028
:1021A0008093910180918E01882319F08150809352
:1021B0008E018091C305882319F081508093C30557
:1021C0008091EC059091ED05A091EE05B091EF05A1
:1021D0000196A11DB11D8093EC059093ED05A09390
:1021E000EE05B093EF058091F905882319F0815031
:1021F0008093F905BF91AF919F918F910F900FBE82
:102200000F901F90189582E083BF81E089BF88BF3F
:1022100008951092340680918E01882301F59AE08A
:1022200090938E0181E08093340680918F01882302
:1022300021F0815080938F01089590938F0183E066
:102240008093340680919001882321F081508093FF
:10225000900108959093900187E08093340608954B
:102260008093C001089599E0699FA001112490E036
:10227000837090709C01220F331F280F391F420F6B
:10228000531F455E5D4F82E0403D580714F04BE11F
:1022900052E0CA0108950F931F93CF93DF93CDB7F8
:1022A000DEB728970FB6F894DEBF0FBECDBFE82F7C
:1022B0000D831E832F8338878093700660933A06C0
:1022C00040933B0681E080935C0638853093C505DA
:1022D0002F812093C4059E819093C6058D818093A4
:1022E000C8059093B8018093B7013093BC01209347
:1022F000BB019093BA018093B901F0E0EE0FFF1F8C
:10230000E05AFF4F0190F081E02D8091EC018111A6
:1023100009958091C50587FF03C08FEF8C8301C0AD
:102320001C828091C4058B838091C6058A8380912D
:10233000C805898369817A818B819C8128960FB633
:10234000F894DEBF0FBECDBFDF91CF911F910F91EB
:102350000895000008950000089500000895000009
:10236000089580913A068823A9F4809143069091BC
:102370004406A0914506B09146062091B9013091DE
:10238000BA014091BB015091BC01820F931FA41F61
:10239000B51FC4C08130A9F48091430690914406D2
:1023A000A0914506B09146062091B9013091BA013D
:1023B0004091BB015091BC01821B930BA40BB50B48
:1023C000ADC0823099F460914306709144068091CB
:1023D0004506909146062091B9013091BA0140918D
:1023E000BB015091BC010E94543A31C08330D9F4F2
:1023F000609143067091440680914506909146068F
:102400002091B9013091BA014091BB015091BC01BA
:102410000E949A3A2093430630934406409345061F
:102420005093460683C08430D9F46091430670917E
:10243000440680914506909146062091B90130915D
:10244000BA014091BB015091BC010E949A3A60933D
:10245000430670934406809345069093460666C0F3
:102460008530A9F48091430690914406A0914506D9
:10247000B09146062091B9013091BA014091BB015B
:102480005091BC0182239323A423B52347C08630F7
:10249000A9F48091430690914406A0914506B0911D
:1024A00046062091B9013091BA014091BB0150918B
:1024B000BC01822B932BA42BB52B30C08730A9F401
:1024C0008091430690914406A0914506B09146063E
:1024D0002091B9013091BA014091BB015091BC01EA
:1024E00082279327A427B52719C0883069F48091E3
:1024F000430690914406A0914506B091460680950A
:102500009095A095B0950AC0893081F48091B90169
:102510009091BA01A091BB01B091BC018093430698
:1025200090934406A0934506B093460680914306D7
:1025300090914406A0914506B09146062091C201B3
:102540003091C3010097A105B10511F4286001C0C5
:10255000277F3093C3012093C201089580913A06EA
:102560008823A9F48091430690914406A0914506E2
:10257000B091460620916C0630916D0640916E0632
:1025800050916F06820F931FA41FB51F16C0813094
:10259000E9F48091430690914406A0914506B091DC
:1025A000460620916C0630916D0640916E06509162
:1025B0006F06821B930BA40BB50B8093430690937D
:1025C0004406A0934506B0934606D8C0823099F4DD
:1025D00060914306709144068091450690914606AD
:1025E00020916C0630916D0640916E0650916F06F9
:1025F0000E94543A31C08330D9F4609143067091FF
:102600004406809145069091460620916C063091D3
:102610006D0640916E0650916F060E949A3A209383
:102620004306309344064093450650934606A6C0A1
:102630008430D9F460914306709144068091450638
:102640009091460620916C0630916D0640916E0681
:1026500050916F060E949A3A609343067093440625
:10266000809345069093460689C08530A9F48091F1
:10267000430690914406A0914506B09146062091EC
:102680006C0630916D0640916E0650916F06822364
:102690009323A423B52391CF8630A9F480914306D8
:1026A00090914406A0914506B091460620916C0693
:1026B00030916D0640916E0650916F06822B932BE0
:1026C000A42BB52B7ACF8730A9F480914306909143
:1026D0004406A0914506B091460620916C063091C3
:1026E0006D0640916E0650916F0682279327A427AE
:1026F000B52763CF883069F480916C0690916D06A0
:10270000A0916E06B0916F0680959095A095B095BA
:102710000AC0893089F48091430690914406A091C3
:102720004506B091460680936C0690936D06A09383
:102730006E06B0936F0622C08A3001F520914306E1
:1027400030914406409145065091460680916C06B2
:1027500090916D06A0916E06B0916F06809343062E
:1027600090934406A0934506B093460620936C06CA
:1027700030936D0640936E0650936F06809143062A
:1027800090914406A0914506B09146062091C20161
:102790003091C3010097A105B10511F4286001C073
:1027A000277F3093C3012093C2010895EF92FF92D7
:1027B0000F931F93E0904306F09044060091450666
:1027C000109146062091B9013091BA014091BB01A8
:1027D0005091BC012E153F05400751073CF48091F4
:1027E000C2019091C30184608C7F0EC08091C201B0
:1027F0009091C301E216F3060407150719F4897FC7
:10280000816002C0887F82609093C3018093C2017F
:102810008091C2019091C301E114F10401051105F9
:1028200011F4886001C0877F9093C3018093C20137
:102830001F910F91FF90EF90089580913A068823A1
:1028400039F48091C2019091C30183FF7AC060C0C6
:10285000813039F48091C2019091C30183FD71C030
:1028600057C0823029F48091C2019091C3012CC0DD
:10287000833039F48091C2019091C30180FD61C021
:1028800047C0843039F48091C2019091C30182FF26
:1028900058C03EC0853039F48091C2019091C30187
:1028A00082FD36C011C0863039F48091C20190910A
:1028B000C30181FF46C02CC0873049F48091C2011A
:1028C0009091C30181FD24C080FF3BC021C08830AE
:1028D00039F48091C2019091C30184FF32C018C0C5
:1028E000893039F48091C2019091C30185FF29C0DC
:1028F0000FC08A3039F48091C2019091C30186FFE4
:1029000020C006C08B3069F48091C20187FF19C0D6
:102910008091B7019091B801909338068093370663
:1029200008958C3071F48091C2019091C30190FFA1
:1029300008C08091B7019091B801909338068093B8
:10294000370608958091B7019091B80190933806A9
:102950008093370608952091A3012830B8F4E22F20
:10296000F0E0EE0FFF1FED56FE4F8091370690917D
:102970003806918380832F5F2093A3018091B70154
:102980009091B80190933806809337060895E091AE
:10299000A301EE2371F0E150E093A301F0E0EE0F0C
:1029A000FF1FED56FE4F80819181909338068093F2
:1029B0003706089580913A06813011F48093920190
:1029C000089580913A06813011F410929201089591
:1029D00010924206089580913A06882339F4809136
:1029E000C2019091C3018F7090701FC0813031F48B
:1029F0008091C2019091C3018F7E17C0823031F463
:102A00008091C2019091C3018F7D0FC0833031F45A
:102A10008091C2019091C3018F7B07C0843051F433
:102A20008091C2019091C3018F779093C3018093ED
:102A3000C2010895853049F48091C2019091C3018B
:102A40009E7F9093C3018093C201089580913A06BE
:102A5000813041F48091C6058093DF018091C805E3
:102A60008093E001089508950000089500000895FE
:102A700000000895000008950000089500000895E2
:102A800000000895000008950000089500000895D2
:102A900000000895000008950000089500000895C2
:102AA00000000895000008950000089500000895B2
:102AB00000000895000008950000089500000895A2
:102AC0000000089500000895000008951092420645
:102AD000089580913A06813041F48091B701909138
:102AE000B801909338068093370681E080934206C0
:102AF000089582E080934206089583E08093420621
:102B000010923806109237068FEF9FEF9093C7010F
:102B10008093C6011092A301109247061092A4015F
:102B200081E08093BF011092C5011092C401109200
:102B300043061092440610924506109246061092E3
:102B40009201089510924F061092C5011092C4018F
:102B5000089580913A068130D9F0813030F082308A
:102B600031F1833009F044C033C080914206809334
:102B7000C505809147068093C4052091C40130911A
:102B8000C501832F99278093C6052093C805089512
:102B9000809142068093C505809147068093C405C5
:102BA000809138068093C605809137060EC08091CB
:102BB00046068093C505809145068093C4058091A3
:102BC00044068093C605809143068093C805089506
:102BD00080916F068093C50580916E068093C40531
:102BE00080916D068093C60580916C068093C80520
:102BF00008958091C80580935D0181E080931C0653
:102C00008091E005882319F082E080931C06809172
:102C10001706882319F083E080931C06089586E048
:102C200080933606089580913A06813049F08130CC
:102C3000A0F0823009F44FC0833009F063C058C05F
:102C40004091DD015091DE016091B7017091B801B2
:102C5000E9ECF1E020E030E03AC02091DD01309174
:102C6000DE012A30310590F4F901EE0FFF1FE75322
:102C7000FE4F8091B7019091B801918380832F5FBF
:102C80003F4F3093DE012093DD01089589E080936A
:102C9000360608958191919186179707B1F4F9014D
:102CA000EE0FFF1FE753FE4F4150504006C02F5F0D
:102CB0003F4F828193818193919324173507B8F315
:102CC0005093DE014093DD0108952F5F3F4F24179D
:102CD000350701F708951092DE011092DD01E9EC4D
:102CE000F1E01192119281E0ED3DF80771F0F9CF1A
:102CF0001092C5051092C4051092C6058AE0809313
:102D0000C805089583E0809336060895809165068E
:102D1000813881F580916606823961F58091670678
:102D2000833A41F580916806843B21F580916906DC
:102D3000853C01F580916A06863DE1F4F894C098DF
:102D4000AB9A89E0E3E0F0E08093570084918670CD
:102D500019F40C9400380895823019F40C94003C56
:102D60000895843019F40C94003E0895863011F4CF
:102D70000C94003F0895CF93DF93CDB7DEB728972B
:102D80000FB6F894DEBF0FBECDBF80913A068130FA
:102D9000F1F480913B068A32C1F48091C8058983A1
:102DA0008091C6058A838091C4058B838091C50577
:102DB0008C831D821E821F821886BE016F5F7F4F2B
:102DC0008FEF97E00E9421312FC084E02BC0882331
:102DD00041F5BE016F5F7F4F8FEF97E00E94EB30B0
:102DE0009091C8058981981799F49091C6058A81B8
:102DF000981771F49091C4058B81981749F49091BC
:102E0000C5058C81981721F481E08093C80502C024
:102E10001092C8051092C5051092C4051092C605FF
:102E200003C083E08093360628960FB6F894DEBF81
:102E30000FBECDBFDF91CF910895809142068823C8
:102E400089F1833079F1853069F165EA71E080912B
:102E50003706909138060E94EB302091370630916A
:102E600038068091C6019091C7018217930721F01F
:102E700081E08093BF0102C01092BF013093C7016F
:102E80002093C6012F5F3F4F3093380620933706BB
:102E900080914206823019F485E08093420681E0F9
:102EA00090E0089580E090E008958CE090E00E942A
:102EB000E60F8093AE0180913A06882399F482E070
:102EC0008093C00124E530E0AEEAB1E0F9018491DD
:102ED000FD0181832F5F3F4F1196F1E0A63BBF07B5
:102EE00061F0F4CF1092C50581E08093C40583E0C2
:102EF0008093C60583E28093C80508952091B701A9
:102F00003091B8013093C5012093C40182E08093D1
:102F1000C0012F5F374078F487E090E00E94E60F11
:102F200080FD09C06FEA71E08091C4019091C501F4
:102F30000E94EB3007C0EEEAF1E0119281E0E73B3E
:102F4000F807D9F78CE090E00E94E60F8093AE017D
:102F5000089583E08093420687E090E00E94E60FA8
:102F600081FD04C081E080934F0603C088E0809318
:102F700036068091B7019091B8019093C501809376
:102F8000C40108950F931F93CF93DF93CDB7DEB79E
:102F900024970FB6F894DEBF0FBECDBFE82FF0E048
:102FA0006623C1F189E0689F800111249F0123708D
:102FB0003070C901880F991F820F931F080F191FC6
:102FC000055E1D4F82E00F3C180744F081E08093BE
:102FD000360660E070E080E090E026C0C80102960E
:102FE0000E94E60F8B83C80101960E94E60FFE0146
:102FF00031968183C8010E94E60F89838B8187FF08
:1030000003C08FEF8C8301C01C8269817A818B8120
:103010009C810AC0EE0FFF1FEE0FFF1FE05BF94F10
:10302000608171818281938124960FB6F894DEBF0E
:103030000FBECDBFDF91CF911F910F910895CF9318
:10304000DF93CDB7DEB724970FB6F894DEBF0FBE7F
:10305000CDBF60913A0680913B060E94C2176983FA
:103060007A838B839C834C814093C5053B8130934D
:10307000C4052A812093C60599819093C805809143
:103080005C068823F9F0409346063093450620936A
:103090004406909343068091430690914406A09184
:1030A0004506B09146062091C2013091C3010097B8
:1030B000A105B10511F4286001C0277F3093C30139
:1030C0002093C20124960FB6F894DEBF0FBECDBF89
:1030D000DF91CF9108958091B7019091B801825D01
:1030E000944041F460E080E090E00E94EE0FF8949C
:1030F0000C94000008950F931F93CF93DF93CDB7E7
:10310000DEB724970FB6F894DEBF0FBECDBF909107
:103110003A06992341F189E0989F8001112480911A
:103120003B0623E0829FC0011124080F191F055E92
:103130001D4F82E00F3C180724F081E08093360693
:1031400032C06091C405C80102960E94EE0F6091E2
:10315000C605C80101960E94EE0F6091C805C8011E
:103160000E94EE0F20C08091C4058B839091C6050C
:103170009A839091C805998387FF03C08FEF8C8352
:1031800001C01C82E0913B06F0E0EE0FFF1FEE0F46
:10319000FF1FE05BF94F89819A81AB81BC818083FD
:1031A0009183A283B38324960FB6F894DEBF0FBE3B
:1031B000CDBFDF91CF911F910F91089590913A0665
:1031C00097FF13C0809146068093C5058091450600
:1031D0008093C405809144068093C6058091430680
:1031E0008093C8059F7790933A0690913A06992369
:1031F00029F0923019F0933009F046C0C39A8BB78A
:1032000080648BBFC49A8BB780648BBF992329F4E9
:103210008BB78F7B8BBFAF980DC0923029F48BB7E3
:103220008F7B8BBFAE9806C0933021F48BB78F7B1A
:103230008BBFAD9880913B06843030F08091C505FE
:103240000E9490108093C50580913B06833030F03A
:103250008091C4050E9490108093C40580913B0624
:10326000823030F08091C6050E9490108093C60590
:103270008091C8050E9490108093C80585B3806E28
:1032800085BB8BB780648BBF80913A06813051F546
:1032900085B3806E85BB8BB780648BBFC49A8BB7B8
:1032A00080648BBF8BB78F7B8BBFC3988091C50524
:1032B0000E9490108093C5058091C4050E949010D3
:1032C0008093C4058091C6050E9490108093C60526
:1032D0008091C8050E9490108093C805C39A8BB74F
:1032E00080648BBF80915C06882359F18091C5056D
:1032F000809346068091C405809345068091C6055B
:10330000809344068091C8058093430680914306CC
:1033100090914406A0914506B09146062091C201C5
:103320003091C3010097A105B10531F428603093B5
:10333000C3012093C2010895277F3093C3012093D6
:10334000C20108951F9381E08093470640913A0699
:10335000442339F08091B7019091B80118161906ED
:1033600004F52091BF01222341F08091B701909193
:10337000B8019093BE018093BD01442391F48091E4
:10338000B7019091B8018F5F9F4F51F5222341F112
:1033900080914306909144069093BE018093BD01B5
:1033A0001FC08091B7019091B801181619061CF042
:1033B00020E030E00AC020E08091BD019091BE0184
:1033C000892B09F021E081E02827122F8091C2018A
:1033D0009091C301222311F0806121C08F7E1FC014
:1033E0008091BD019091BE01892B11F41092470686
:1033F00080914706882341F08091C6019091C701D2
:1034000090933806809337068091C2019091C30152
:103410008F7E9093C3018093C20110E025C09093EA
:10342000C3018093C2014130F9F460E08DE70E944E
:10343000EB0790E020913B06220F02C095958795FF
:103440002A95E2F780FF02C0109247068091470656
:10345000882351F0112341F48091C6019091C70156
:10346000909338068093370680913A06823019F59A
:1034700063E08DE70E94EB0790E040913B06440F2C
:1034800022E030E002C0220F331F4A95E2F7822388
:103490009323892B11F010924706809147068823C9
:1034A00051F0112341F48091C6019091C70190938E
:1034B00038068093370680913A068330F9F463E04A
:1034C0008DE70E94EB0790E020913B06220F02C09F
:1034D000959587952A95E2F780FF02C010924706DE
:1034E00080914706882351F0112341F48091C60151
:1034F0009091C701909338068093370680913A06E1
:10350000843009F049C0E0913B06E33050F410925A
:103510004706F0E0E051FA4F8081882379F181E09D
:1035200028C0E43049F48091F005882301F520E0BB
:1035300030E08091F10515C0E53059F0E63019F41E
:103540008091F00508C0E730B9F48091F005882338
:1035500071F48091F105882351F420E030E08091EE
:10356000F205882311F021E030E0C90102C081E0BA
:1035700090E08093470602C010924706809147066C
:10358000882351F0112341F48091C6019091C70125
:1035900090933806809337061F91089580913A06DC
:1035A000882341F4E0913B06F0E0E051FA4F81E0DE
:1035B00080830895813081F480913B06E82FF0E00C
:1035C000E051FA4F9FE0908362E00E94E40880910E
:1035D0003B060E9436090895823049F5E0913B068A
:1035E000F0E0E051FA4FE081E093C80580915C067D
:1035F0008823E9F08E2F90E0A0E0B0E080934306AE
:1036000090934406A0934506B09346068091C2016C
:103610009091C301EE2331F488609093C3018093AD
:10362000C2010895877F9093C3018093C2010895DA
:1036300062E080913B060E94E40880913B060E9474
:1036400036090895EF92FF920F931F93CF93DF9364
:1036500080913B06882341F480913A06873109F036
:1036600001C10E949C09FEC0813009F0B0C0809168
:103670003A06863038F4C82FD0E0C759DE4F833081
:10368000E1F415C0893038F4C82FD0E0CC0FDD1F2D
:10369000CC59DE4F12C08C3008F0E1C0C82FD0E00A
:1036A000CC0FDD1FCC0FDD1FCC5ADE4F06C0CE0184
:1036B0000E94E60F8093C7040FC0843031F4CE011E
:1036C0000E94E60F8093C60407C0853029F4CE011E
:1036D0000E94E60F8093C80480913A06863061F418
:1036E000CE0101960E94E60F8093CA04CE010E948B
:1036F000E60F8093C904B6C0873061F4CE0101960D
:103700000E94E60F8093C304CE010E94E60F8093CF
:10371000C204A8C0883061F4CE0101960E94E60F71
:103720008093C504CE010E94E60F8093C4049AC022
:103730008930C1F4CE0103960E94E60F8093B00554
:10374000CE0102960E94E60F8093AF05CE0101964E
:103750000E94E60F8093AE05CE010E94E60F809393
:10376000AD0580C08A30C1F4CE0103960E94E60FF9
:103770008093B405CE0102960E94E60F8093B305B4
:10378000CE0101960E94E60F8093B205CE010E9401
:10379000E60F8093B10566C08B3009F063C0CE019F
:1037A00003960E94E60F8093C104CE0102960E9408
:1037B000E60F8093C004CE0101960E94E60F80932D
:1037C000BF04CE010E94E60F8093BE044BC082303E
:1037D00009F048C000913A06083308F043C010E0F1
:1037E000000F111F000F111FBBE1EB2EB3E0FB2EEA
:1037F000E00EF11EC7010E94E60F04531B4FF801B3
:10380000808380913A06C82FD0E0CC0FDD1FCC0F0B
:10381000DD1FC353DB4FC70101960E94E60F88836B
:1038200080913A06C82FD0E0CC0FDD1FCC0FDD1FF2
:10383000C253DB4FC70102960E94E60F8883809136
:103840003A06C82FD0E0CC0FDD1FCC0FDD1FC153CF
:10385000DB4FC70103960E94E60F888303C0CFEFBA
:10386000D3E02BCFDF91CF911F910F91FF90EF907D
:1038700008950F931F93CF93DF9380913B06882386
:1038800021F480913A06893449F089E090E00E9461
:10389000E60F882319F085E08093360680913B0679
:1038A000882311F580913A06803428F5873088F412
:1038B000863011F48EE70AC0880F880F8C590E9459
:1038C000D30A80913A06880F880F8A590E94D30A3A
:1038D000F0C0873019F40E94920AEBC0873109F0DA
:1038E000E8C00E94510AE5C0813009F09FC0809174
:1038F0003A06833020F483E080933606DAC08630BF
:1039000038F4C82FD0E0C759DE4F8330C9F415C052
:10391000893038F4C82FD0E0CC0FDD1FCC59DE4FF2
:103920000FC08C3008F0C2C0C82FD0E0CC0FDD1F14
:10393000CC0FDD1FCC5ADE4F03C06091C70409C015
:10394000843019F46091C60404C0853029F4609174
:10395000C804CE010E94EE0F80913A06863049F4E9
:103960006091CA04CE0101960E94EE0F6091C904D5
:103970005BC0873049F46091C304CE0101960E9478
:10398000EE0F6091C20450C0883049F46091C504C4
:10399000CE0101960E94EE0F6091C40445C08930AB
:1039A000A9F46091B005CE0103960E94EE0F6091DC
:1039B000AF05CE0102960E94EE0F6091AE05CE01DA
:1039C00001960E94EE0F6091AD052EC08A30A9F4D9
:1039D0006091B405CE0103960E94EE0F6091B3058D
:1039E000CE0102960E94EE0F6091B205CE010196C3
:1039F0000E94EE0F6091B10517C08B3009F059C0DD
:103A00006091C104CE0103960E94EE0F6091C00444
:103A1000CE0102960E94EE0F6091BF04CE01019686
:103A20000E94EE0F6091BE04CE013DC0823009F0CD
:103A300040C0E0913A06E833E0F5F0E0EE0FFF1FFA
:103A4000EE0FFF1F8F01055E1C4FE453FB4F638198
:103A5000C80103960E94EE0FE0913A06F0E0EE0FE7
:103A6000FF1FEE0FFF1FE453FB4F6281C801029658
:103A70000E94EE0FE0913A06F0E0EE0FFF1FEE0F0E
:103A8000FF1FE453FB4F6181C80101960E94EE0FB6
:103A9000E0913A06F0E0EE0FFF1FEE0FFF1FE45338
:103AA000FB4F6081C8010E94EE0F03C0CFEFD3E04F
:103AB00047CFDF91CF911F910F9108950F931F93DF
:103AC000CF93DF93CDB7DEB728970FB6F894DEBF5C
:103AD0000FBECDBF80913B06882309F007C18091BE
:103AE0003A0687FDA8C0803408F041C08630A9F4AA
:103AF0008FE78093D80561EE75E088ED95E00E9430
:103B0000BC048091E4058093C8058091E30580930F
:103B1000C6058091E2058093C40580913A068730FE
:103B200008F474C1880F880F8B598093D80561EE13
:103B300075E088ED95E00E94BC048091E4058093D7
:103B4000C8058091E3058093C6058091D8058E5FF6
:103B50008093D80561EE75E088ED95E00E94BC0485
:103B60008091E4058093C4058091E30561C08035B0
:103B700019F406E010E012C0813519F407E010E0F6
:103B80000DC0823519F409E112E008C0082F10E0D9
:103B900000541040833511F405E112E01092C6057F
:103BA000C8010E94E60F8093C80590913A06892FBC
:103BB00086548230F0F4963419F40EE411E002C019
:103BC0000AE411E0C8010E94E60F8093C805C8010D
:103BD00001960E94E60F8093C605C80102960E94D6
:103BE000E60F8093C405C80103960E94E60F8093F8
:103BF000C50580913A06823531F4C80101960E94CC
:103C0000E60F8093C60580913A06833509F0FEC021
:103C1000C80101960E94E60F8093C605C80102966E
:103C20000E94E60F8093C405C80103960E94E60F28
:103C30008093C505EBC01092C5051092C405109283
:103C4000C605803819F48091420616C0813819F4EF
:103C500080914F0611C0823859F4809137069091B7
:103C60003806892F99278093C6058091370604C0AE
:103C7000833829F48091A4018093C8052FC084382B
:103C8000C9F4F8948091EC059091ED05A091EE05B2
:103C9000B091EF0589839A83AB83BC837894898143
:103CA0008093C8058A818093C6058B818093C40563
:103CB0008C8112C0853891F40E94463A6D837E83D0
:103CC0008F8398878D818093C8058E818093C605E8
:103CD0008F818093C40588858093C50580913A06BD
:103CE0008F3F09F093C08091C1018EC0813009F0EF
:103CF00074C01092C5051092C4051092C60580913B
:103D00003A06882319F48091CB0415C08130A9F0BC
:103D1000823019F48091AC050EC0833019F4809183
:103D2000C70409C0843019F48091C60404C08530EA
:103D300021F48091C8048093C80580913A068630AA
:103D400039F48091CA048093C6058091C9045CC08F
:103D5000873039F48091C3048093C6058091C204F2
:103D600053C0883039F48091C5048093C605809192
:103D7000C4044AC0893079F48091B0058093C505A8
:103D80008091AF058093C4058091AE058093C605F0
:103D90008091AD0539C08A3079F48091B405809363
:103DA000C5058091B3058093C4058091B2058093C9
:103DB000C6058091B10528C08B3041F58091C104C2
:103DC0008093C5058091C0048093C4058091BF0491
:103DD0008093C6058091BE0417C08230B9F4E0918B
:103DE0003A06E83398F4F0E0EE0FFF1FEE0FFF1FE6
:103DF000E453FB4F83818093C50582818093C40582
:103E000081818093C60580818093C80580915C067E
:103E1000882339F18091C505809346068091C405B9
:103E2000809345068091C605809344068091C8051D
:103E3000809343068091430690914406A0914506E5
:103E4000B09146062091C2013091C3010097A105AF
:103E5000B10511F4286001C0277F3093C30120937E
:103E6000C20128960FB6F894DEBF0FBECDBFDF911A
:103E7000CF911F910F910895AF92BF92CF92DF9291
:103E8000EF92FF920F931F9380913B06882309F0D6
:103E90006BC180913A0687FD35C1803458F5863074
:103EA00061F42091C805207F6091C4056F7C606239
:103EB0004091C6058EE70E94A00500913A060730A2
:103EC00008F402C210E0000F111F000F111F209113
:103ED000C8054091C60560E0802F8C590E94A0055E
:103EE0002091C4054091C50560E0802F8A590E9449
:103EF000A005EAC1893409F58091B7019091B80114
:103F000024E0823D920731F41092C60581E080934F
:103F1000C8050CC0815E904129F41092C60510922C
:103F2000C80504C084E080933606CEC16091C80500
:103F300089E090E00E94EE0FC7C1803519F406E0D9
:103F400010E015C0813529F0082F10E00054104012
:103F50000EC08091C80580FD08C087E090E00E94F7
:103F6000E60F80FF02C00E946F3007E010E08091F2
:103F70003A06823581F48091B7019091B80190930F
:103F8000D7058093D6056091C6058AE192E00E942C
:103F9000EE0F09E112E080913A068335A1F46091B9
:103FA000C50588E192E00E94EE0F6091C40587E1AB
:103FB00092E00E94EE0F6091C60586E192E00E94B9
:103FC000EE0F05E112E080913A06873419F40AE415
:103FD00011E004C0863411F40EE411E086548230FE
:103FE00090F46091C505C80103960E94EE0F6091A0
:103FF000C405C80102960E94EE0F6091C605C80173
:1040000001960E94EE0F6091C805C8010E94EE0F54
:1040100080913A06873429F0853419F0833509F008
:104020004BC08AE491E00E94E60F809330068BE457
:1040300091E00E94E60F809331068CE491E00E94AB
:10404000E60F809332068DE491E00E94E60F8093A4
:10405000330685E192E00E94E60F8093DC0586E15D
:1040600092E00E94E60F8093DD0587E192E00E94D6
:10407000E60F8093DE0588E192E00E94E60F8093D0
:10408000DF05E090DC05F090DD050091DE05109184
:10409000DF05A0903006B0903106C0903206D09077
:1040A000330685E090E00E94E60F98018701B60193
:1040B000A50190E00E94BA3480913A068634C1F49A
:1040C0008EE491E00E94E60F8093E8058FE491E092
:1040D0000E94E60F8093E90580E591E00E94E60FDB
:1040E0008093EA0581E591E00E94E60F8093EB055D
:1040F00080913A06823409F0E7C08091C8050E9499
:104100001038E2C0833829F48091C8058093A40157
:1041100021C0843899F4F8948091B9019091BA0142
:10412000A091BB01B091BC018093EC059093ED058B
:10413000A093EE05B093EF0578940CC0853851F448
:104140006091B9017091BA018091BB019091BC015D
:104150000E944B3A80913A068F3F09F0B5C080919A
:10416000C8058093C101B0C0813009F094C080912E
:104170003A06882329F48091C8058093CB04A4C013
:10418000813009F44FC0823029F48091C8058093B2
:10419000AC059AC0833029F48091C8058093C70488
:1041A00093C0843029F48091C8058093C6048CC0E4
:1041B000853029F48091C8058093C80485C0863075
:1041C00079F48091C60590E0982F88272091C80542
:1041D00030E0822B932B9093CA048093C90474C05F
:1041E000873079F48091C60590E0982F8827209138
:1041F000C80530E0822B932B9093C3048093C204B4
:1042000063C0883079F48091C60590E0982F8827A4
:104210002091C80530E0822B932B9093C5048093A6
:10422000C40452C0893089F48091B9019091BA01D7
:10423000A091BB01B091BC018093AD059093AE05F8
:10424000A093AF05B093B0053FC08A3089F4809148
:10425000B9019091BA01A091BB01B091BC018093CA
:10426000B1059093B205A093B305B093B4052CC0EB
:104270008B3051F58091B9019091BA01A091BB01A9
:10428000B091BC018093BE049093BF04A093C0047E
:10429000B093C10419C08230B9F4E0913A06E83312
:1042A00098F4F0E0EE0FFF1FEE0FFF1FE453FB4FFB
:1042B0008091C50583838091C40582838091C60562
:1042C00081838091C80580831F910F91FF90EF90AB
:1042D000DF90CF90BF90AF90089530914606309315
:1042E000C505209145062093C405909144069093FE
:1042F000C605809143068093C8059093B8018093CA
:10430000B7013093BC012093BB019093BA01809315
:10431000B9010E943C1F08950F931F93CF93DF9321
:10432000E0913A06E7FD08C0EF3008F0B9C0F0E0D0
:10433000E059FE4FE49101C0EF77E0933A06909187
:104340003A069034C8F4E92FF0E000913B069F3024
:1043500040F4EE0FFF1F0295000F007E802F8E2B82
:1043600008C0EB5AFE4F8491880F0295000F007E23
:10437000802B0E941D0B94C09B34E1F480913B067E
:10438000C82FD0E0CC0FDD1FCE01865A9E4F0E9471
:10439000E60FCF5ED94F888380913B06C82FD0E0CF
:1043A000CC0FDD1FCE01855A9E4F0E94E60FCF5ED7
:1043B000D94F1DC09C34E9F480913B06C82FD0E052
:1043C000CC0FDD1FCE01805A9E4F0E94E60FCD50CC
:1043D000DA4F888380913B06C82FD0E0CC0FDD1FD9
:1043E000CE018F599E4F0E94E60FCD50DA4F898340
:1043F00057C09335E1F480913B06C82FD0E0CC0F35
:10440000DD1FCE018A599E4F0E94E60FC95ADE4F2A
:10441000888380913B06C82FD0E0CC0FDD1FCE01F2
:1044200089599E4F0E94E60FC95ADE4FE0CF892F6F
:104430008155823020F483E08093360631C00091AC
:104440003B069D3459F410E0C80183509C4F0E94F4
:10445000E60F085E194FF801808322C0C02FD0E01C
:10446000C05CD04083E0989FC0011124C80FD91FC1
:10447000CE0140960E94E60F8093C805682F8C2FCE
:104480000E94741080913A06853451F4CE010D9645
:104490000E94E60F682F9E012350822F0E94741005
:1044A000DF91CF911F910F9108951F93CF93DF93C9
:1044B000E0913A06E7FD08C0EF3008F0B3C0F0E045
:1044C000E059FE4FE49101C0EF77E0933A06209166
:1044D0003A062034D0F4E22FF0E090913B062F30E2
:1044E00040F4EE0FFF1F9295990F907E892F8E2B2F
:1044F00008C0EB5AFE4F8491880F9295990F907ED9
:10450000892B0E94D30A182F88C02B34C9F48091BC
:104510003B0690E0880F991FFC01EF5EF94F608128
:10452000865A9E4F0E94EE0F80913B0690E0880FC6
:10453000991FFC01EF5EF94F6181855A9E4F1AC0A9
:104540002C34D9F480913B0690E0880F991FFC0130
:10455000ED50FA4F6081805A9E4F0E94EE0F80917D
:104560003B0690E0880F991FFC01ED50FA4F6181E6
:104570008F599E4F0E94EE0F55C02335C9F480918C
:104580003B0690E0880F991FFC01E95AFE4F6081BD
:104590008A599E4F0E94EE0F80913B0690E0880F53
:1045A000991FFC01E95AFE4F618189599E4FE2CF64
:1045B0002D3451F480913B0690E0FC01E85EF94F08
:1045C000608183509C4FD6CF822F8155823010F46A
:1045D00083E026C080913B06C82FD0E0C05CD0406D
:1045E00083E0289FC0011124C80FD91F8C2F0E947F
:1045F0006D10682FCE0140960E94EE0F182F80910B
:104600003A06853451F49E012350822F0E946D108A
:10461000682FCE010D960E94EE0F123019F485E03E
:1046200080933606DF91CF911F910895DF92EF922C
:10463000FF920F931F93CF93DF93CDB7DEB72697EB
:104640000FB6F894DEBF0FBECDBFE0913A06E7FD8E
:1046500008C0EF3008F007C2F0E0E059FE4FE491E7
:1046600001C0EF77E0933A0620913A062B3108F02B
:10467000B3C0233041F4E0913B06F0E0EE0FFF1FA2
:10468000E25AF94F09C0263061F4E0913B06F0E0B0
:10469000EE0FFF1FE85BF94F81818093C605808193
:1046A00090C090913B06E22FF0E0293058F5EE0FD4
:1046B000FF1F9295990F907E9E2B91609093D80545
:1046C00061EE75E088ED95E00E94BC048091E20502
:1046D0008093C4059091E3059093C6058091E4050D
:1046E0008093C80580913A06843008F46CC093FF2B
:1046F0006AC0906F9093C6058FEF8093C405809336
:10470000C50561C0EB5AFE4F8491880F9295990FB1
:10471000907E982B91609093D80561EE75E088EDBE
:1047200095E00E94BC041E828091E2058D838091F9
:10473000E3058C838091E4058B832B813C814D8143
:104740005E81E0913A068E2F90E0FC01ED5BFE4F1A
:10475000E49104C05595479537952795EA95D2F78A
:104760002B833C834D835E83815D9E4FEE24FF242B
:10477000870160E070E0FC01D4900FC081E090E020
:10478000A0E0B0E004C0880F991FAA1FBB1FEA95E4
:10479000D2F7E82AF92A0A2B1B2BE62F6F5F7F4FEF
:1047A000ED1560F3E222F32204231523EB82FC8251
:1047B0000D831E838D818093C4058C818093C605F3
:1047C0008B818093C8058091C40587FF02C08FEF5D
:1047D0001DC11092C5051CC12E3108F03FC01092BA
:1047E000C5051092C4051092C6051092C8058DE744
:1047F0008093D80561EE75E088ED95E00E94BC04D9
:1048000080913A068B3199F480913B06880F22E023
:1048100030E002C0220F331F8A95E2F78091E40551
:1048200090E028233923232B09F4F2C015C08C31E2
:1048300019F48091E40505C08D3109F0E9C080913B
:10484000E10590E020913B06220F02C095958795E7
:104850002A95E2F780FFDCC081E098C0203408F49C
:10486000D7C0203608F095C010913B06105C83E05D
:10487000289FC0011124180F253431F4812F835053
:104880000E946D108093C605812F0E946D10809349
:10489000C80580913A068B34A9F4E0913B06F0E01C
:1048A000EE0FFF1FEF5EF94F91819093C605808157
:1048B0008093C80597FF1FC08FEF8093C505809335
:1048C000C40519C08C3441F4E0913B06F0E0EE0FD2
:1048D000FF1FED50FA4F09C0833569F4E0913B06A4
:1048E000F0E0EE0FFF1FE95AFE4F81818093C6056D
:1048F00080818093C80580913A068D3431F4E0912F
:104900003B06F0E0E85EF94F0FC08E3431F4E091E1
:104910003B06F0E0EB51FA4F07C0803541F4E091DF
:104920003B06F0E0E250FA4F80818093C805809109
:104930003A068135A1F480913B060E94B2396B831F
:104940007C838D839E838E818093C5058D8180932A
:10495000C4058C818093C6058B818093C8058091A6
:104960003A06873419F0803409F052C09091C80596
:1049700084E6989FC001112461E170E00E94733ABF
:104980007A8369838A818093C60589818093C8056B
:104990003FC02236C1F41092C605E0913B06F0E01C
:1049A000E15CF94F808181FF04C081E08093C805FC
:1049B00002C01092C805E0913B06F0E0E15CF94FBF
:1049C00080818D7F808380913A068336C1F4109276
:1049D000C605E0913B06F0E0E15CF94F808182FF83
:1049E00004C081E08093C80502C01092C805E09120
:1049F0003B06F0E0E15CF94F80818B7F8083809102
:104A0000C60587FF05C08FEF8093C4058093C50559
:104A100080915C06882339F18091C5058093460614
:104A20008091C405809345068091C6058093440615
:104A30008091C80580934306809143069091440677
:104A4000A0914506B09146062091C2013091C30164
:104A50000097A105B10511F4286001C0277F3093AC
:104A6000C3012093C20126960FB6F894DEBF0FBE95
:104A7000CDBFDF91CF911F910F91FF90EF90DF900D
:104A800008950F931F93CF93DF93982FC82FDD279F
:104A9000C7FDD095FE01E45CF94F8081882319F4AD
:104AA00080E090E01EC010828E01000F111FF801FF
:104AB000E85BF94F60817181892F0E945808025A82
:104AC000194F25E0CC0FDD1F2A95E1F7F801208171
:104AD000418160E0FE01E6608E2F0E94A00581E02A
:104AE00090E0DF91CF911F910F910895CF93DF93C5
:104AF000CDB7DEB722970FB6F894DEBF0FBECDBF9D
:104B000090913B06E92FF0E0E45CF94F8081813021
:104B100019F4892F0E9441258091B7019091B80125
:104B2000909581959F4F9A83898362E080913B069F
:104B30000E94E40880913B068295880F807E29813F
:104B40004A8160E088600E94A00580913B068295C2
:104B5000880F807E2FEF47E060E086600E94A0050E
:104B6000E0913B06F0E0E45CF94F82E0808322961E
:104B70000FB6F894DEBF0FBECDBFDF91CF91089581
:104B800090913B06E92FF0E0E45CF94F80818130A1
:104B900019F4892F0E94412562E080913B060E9412
:104BA000E40880913B068295880F807E2091C8059D
:104BB0004091C60560E088600E94A00580913B0698
:104BC0008295880F807E2FEF47E060E086600E942C
:104BD000A005E0913B06F0E0E45CF94F82E08083C1
:104BE0000895DF92EF92FF920F931F93CF93DF937D
:104BF000CDB7DEB724970FB6F894DEBF0FBECDBF9A
:104C0000D62E082F10E0C801E5E0880F991FEA951D
:104C1000E1F782600E9429089B01AC01DD2069F167
:104C20007801EE0CFF1CE00EF11E8BE192E0E80E25
:104C3000F91E89E0D89EC0011124E80EF91E9FECF0
:104C4000E91692E0F90624F081E08093360620C050
:104C500029833A834B835C836B81C70102960E9450
:104C6000EE0FFE0131966181C70101960E94EE0FA1
:104C70006981C7010E94EE0F0BC0000F111F000FCA
:104C8000111F005B194FF801208331834283538346
:104C900024960FB6F894DEBF0FBECDBFDF91CF9143
:104CA0001F910F91FF90EF90DF9008951F93109147
:104CB0003A0680913B06833010F4612F30C0843077
:104CC00041F4612F80E00E94F125612F81E00E9474
:104CD000F12580913B06853041F4612F81E00E94EF
:104CE000F125612F82E00E94F12580913B068630FC
:104CF00041F4612F80E00E94F125612F82E00E9443
:104D0000F12580913B06873061F4612F80E00E949D
:104D1000F125612F81E00E94F125612F82E00E9440
:104D2000F1251F910895CF92DF92EF92FF920F939A
:104D30001F93182F062F8295880F807E82600E9415
:104D400029086B017C01602F812F0E94C2176C150E
:104D50007D058E059F0529F460E070E080E090E01D
:104D600010C0C616D706E806F9062CF46C197D09A2
:104D70008E099F0906C0C61AD70AE80AF90AC701B0
:104D8000B6011F910F91FF90EF90DF90CF900895A3
:104D90000F931F93182F062F60E00E94E408602FE6
:104DA000812F0E94C217AB01BC01812F8295880F11
:104DB000807E0E9400091F910F9108954F925F928B
:104DC0006F927F928F929F92AF92BF92CF92DF921B
:104DD000EF92FF920F931F93CF93DF93CDB7DEB780
:104DE00028970FB6F894DEBF0FBECDBF4091C50522
:104DF00048872091C4052F833091C6053E8380915A
:104E0000C8058D83E0913A06E7FD08C0EF3008F051
:104E100096C1F0E0E059FE4FE49101C0EF77E093D6
:104E20003A06E0913A06E73411F0E03479F48091E3
:104E3000B7019091B80153E0880F991F5A95E1F797
:104E40006FE270E00E94873A6093C805E03408F092
:104E5000E8C0E930B0F5E63081F46091B7017091B7
:104E6000B80180913B060E945808E0913B06F0E0B3
:104E7000EE0FFF1FE85BF94FDDC02093D90530939B
:104E8000DA058091C8058093DB05EE0F80913B0623
:104E90008295880F807E8E2B8093D80561EE75E019
:104EA00088ED95E00E94BC0480913A06833009F0B9
:104EB0003AC1E0913B06F0E0EE0FFF1FE25AF94FD6
:104EC000B9C0E031E9F480913B068295880F807E7D
:104ED00081618093D80561EE75E088ED95E00E94D0
:104EE000BC0480913B068295880F807E8061809310
:104EF000D8059091C8059F708091E205807F1FC002
:104F000090913B06E13169F59295990F907E916100
:104F10009093D80561EE75E088ED95E00E94BC04A1
:104F200080913B068295880F807E80618093D805B2
:104F30009091C8059295907F8091E2058F70982B93
:104F40009093D9058091E3058093DA058091E4057B
:104F50008093DB0561EE75E088ED95E00E94BC046E
:104F6000E2C01C822B833A838091C8058983F0E0DC
:104F7000EB5AFE4FE491EE0FB92EB294BB0C90EEBB
:104F8000B922BE2A8B2D0E942908AB01BC01E091F9
:104F90003A068E2F90E0FC01ED5BFE4FE49101E0BC
:104FA00010E020E030E004C0000F111F221F331F6B
:104FB000EA95D2F7C980DA80EB80FC80442455243E
:104FC000815D9E4FFC01A49025C03601470104C0BD
:104FD00095948794779467948A95D2F7D401C30106
:104FE00081709070892B29F0402B512B622B732BF1
:104FF0000AC0D901C80180959095A095B095482325
:1050000059236A237B23000F111F221F331F08948B
:10501000411C511C842D4A14C0F28B2D0E940009A2
:1050200082C0EB3471F4E0913B06F0E0EE0FFF1F1D
:10503000EF5EF94F8091B7019091B8019183808321
:1050400072C0EC3441F4E0913B06F0E0EE0FFF1F3C
:10505000ED50FA4FEFCFE33541F4E0913B06F0E03D
:10506000EE0FFF1FE95AFE4FE5CFED3449F4E09112
:105070003B06F0E0E85EF94F8091C805808353C09D
:10508000E13579F44C832B833A838091C805898379
:1050900049815A816B817C8180913B060E94EF3867
:1050A00042C0E235C1F44C832B833A838091C8051A
:1050B000898369817A818B819C81462F4F71F5E0CC
:1050C0009595879577956795FA95D1F780913B06E9
:1050D0000E94153928C0E03630F510913B06105C6F
:1050E00083E0E89FC0011124180FE53429F4632FF1
:1050F000812F83500E9474106091C805812F0E94F7
:10510000741080913B068B5E0E946D10682F809119
:105110003B060E94B50F80913A06873411F0803427
:1051200011F41092C60588858093C5058F81809300
:10513000C4058E818093C6058D818093C80528960D
:105140000FB6F894DEBF0FBECDBFDF91CF911F9198
:105150000F91FF90EF90DF90CF90BF90AF909F9016
:105160008F907F906F905F904F900895309146069A
:105170003093C505209145062093C40590914406BF
:105180009093C605809143068093C8059093B8011B
:105190008093B7013093BC012093BB019093BA0177
:1051A0008093B9010E94DE2608951092C5051092E1
:1051B000C4051092C60580913B06882331F5809185
:1051C0003A06883018F40E94800F1DC08A30A0F47F
:1051D0000E94B20F90E020913A0630E02850304013
:1051E00002C0959587952A95E2F780FF02C081E07D
:1051F0000AC01092C80509C083B390E096958795C0
:105200009695879581708093C80580913B06813083
:1052100081F4E0913A06F0E0EE0FFF1FEF5FF94FE7
:1052200020813181818183708093C6052093C805D8
:1052300008C0823031F480913A060E94A40F809316
:10524000C80580915C06882359F18091C50580933B
:1052500046068091C405809345068091C6058093DB
:1052600044068091C805809343068091430690913F
:105270004406A0914506B09146062091C2013091A6
:10528000C3010097A105B10531F428603093C30133
:105290002093C2010895277F3093C3012093C20158
:1052A000089580913B06882339F46091C805809168
:1052B0003A060E948A0F0895823071F48091C805E1
:1052C00080FF05C080913A060E94780F0895809172
:1052D0003A060E947C0F08958F3F21F56091C80522
:1052E00080E00E9419056091C60581E00E941905C1
:1052F0006091C40582E00E9419058091C80582FF73
:1053000003C080E00E9436098091C60582FF03C079
:1053100081E00E9436098091C40582FF03C082E0CB
:105320000E94360908950F931F93CF93DF93CDB753
:10533000DEB72F970FB6F894DEBF0FBECDBF8091BA
:10534000B50590913F06892B80933F0680914006DA
:105350009091B605892B809340068091B705909176
:105360004106892B8093410680911B06882349F0D2
:105370008091C2019091C30191609093C301809389
:10538000C2018091340680FF0BC08091BD019091D5
:10539000BE01009729F001979093BE018093BD0153
:1053A0000E94DD09282F8093EB014091E901509183
:1053B000EA014130510519F0882309F483C0309186
:1053C000E005832F8150823010F02230E1F580918A
:1053D000E8059091E905A091EA05B091EB058C8371
:1053E0009D83AE83BF831A821B822230C1F031308D
:1053F00011F497E001C098E0EFEAF1E0DE011896C1
:1054000081918D9321E0E73BF207D1F79983CE019B
:1054100001960E94CE36882309F450C222C0EFE1E3
:10542000F6E0DE01189681918D9386E0E732F80769
:10543000D1F787E08983CE0101960E94CE3688237A
:1054400009F43CC23CC080911706882319F423302C
:1054500091F40DC0233059F068E08FEA91E00E948A
:105460003A388091E9019091EA018E7F23C268E089
:105470008FE196E0F4CF8091F905882309F01EC2F0
:10548000213091F04E7F5093EA014093E9010EEAFA
:1054900011E0F80181918F010E941430F1E0073B87
:1054A0001F0709F40BC2F5CF0EE116E0F801819158
:1054B0008F010E941430F6E007321F07B9F71092EF
:1054C000EB01FCC11092C80184E696E00E94E90657
:1054D000813069F58093C8018091640680937006DD
:1054E0008091650680933A068091660680933B061C
:1054F000809167068093C505809168068093C405F6
:10550000809169068093C60580916A068093C805DC
:1055100080914206882319F481E090E053C020E096
:1055200030E0833011F421E030E0C9014BC08091BC
:10553000340682FF23C080914206813009F044C0C6
:1055400090919201913009F03FC083E08093C801AF
:1055500087E18093700610923A0610923B061092F3
:10556000C5051092C4058091DF018093C605809126
:10557000E0018093C80590935C0626C00E941D1729
:10558000882311F182E08093C8018091A501809366
:1055900070068091A60180933A068091A7018093BE
:1055A0003B068091A8018093C5058091A901809355
:1055B000C4058091AA018093C6058091AB018093B8
:1055C000C80581E080935C068091C801882309F4B6
:1055D00075C182E090E00E94E60F382F80934E065E
:1055E0002091C6052093B8019091C8059093B7010A
:1055F0008091C5058093BC018091C4058093BB0157
:105600002093BA019093B9011092360690917006DA
:10561000892F8854883310F09E3870F08091C8012B
:10562000813011F4923F41F082E080933606809100
:10563000A40181608093A4018091C801813091F41C
:10564000E4E6F6E08191380F26E0EB36F207D1F779
:1056500030934E0680916B063817C9F081E0809335
:10566000360615C0823099F4E5EAF1E08191380FF1
:1056700081E0EC3AF807D1F730934E068091AC0107
:10568000381729F08091A40182608093A4011092C0
:10569000C00180913606882309F095C080914F069D
:1056A000882311F097FF50C0923F21F40E94861684
:1056B00082E087C0E92FF0E097FF05C0EE0FFF1FE3
:1056C000E051F04004C0EE0FFF1FE05AFF4F019081
:1056D000F081E02D84E6809336068091EC018823EA
:1056E00011F0099503C08FEF809336066091DD01BC
:1056F0007091DE016115710509F465C08091420663
:10570000813009F060C08091C801823009F05BC02F
:10571000409137065091380620E030E00FC02F5FEF
:105720003F4FEE0FFF1FE753FE4F808191814817D7
:10573000590721F485E08093420645C0E22FF0E04E
:10574000E617F70760F33FC08091C4019091C5014F
:10575000E7E08F3F9E07A0F564E676E00E942131E6
:10576000882371F561EE71E08091C4019091C501CB
:105770000E94EB3085E68093360620E030E0F901A8
:10578000EF51FE4FD901AC59B94F90818C919817C8
:1057900021F087E08093360605C02F5F3F4F283009
:1057A000310569F780913606853669F48091C40128
:1057B0009091C50101969093C5018093C40103C0E7
:1057C00087E0809336068091C801813009F076C069
:1057D0008CE090E00E94E60F182F82E090E00E949B
:1057E000E60F282F809339068091C0018823C9F5E0
:1057F00090917006963031F48091C405880F880B23
:105800008093C5051093AE012093AF0180913606B9
:105810008093B0019093B1018091C5058093B2014E
:105820008091C4058093B3018091C6058093B40133
:105830008091C8058093B50180911706882339F0BF
:1058400010924E0690914E06EFEAF1E003C01093DD
:105850004E06F8CF8191980F21E0E63BF207D1F791
:105860000FC0813089F41093AE0110924E06EEEA1B
:10587000F1E090E08191980F81E0E63BF807D1F7E5
:1058800090934E069093B6018BE090E00E94E60F55
:105890008093F9058091C101882351F080917006B1
:1058A000863031F08A3021F08F3011F08F3131F4B1
:1058B00081E090E09093EA018093E9012F960FB682
:1058C000F894DEBF0FBECDBFDF91CF911F910F9136
:1058D00008959F92AF92BF92CF92DF92EF92FF9284
:1058E0000F931F93CF93DF93CDB7DEB722970FB6F9
:1058F000F894DEBF0FBECDBF6C017B01042F611594
:10590000710509F499C0009709F496C068177907E2
:1059100009F492C0142F1295110F107EA6E09A2E52
:10592000912A892D0E940F089A838983812F8C6088
:105930000E940F085C0180E0D7FC07C0EE0CFF1C42
:10594000CC0CDD1C8F5F8F30B9F7E114F10419F432
:1059500071E0E72EF12C40E050E001C07901142FF6
:105960004F5F5F4FC70180709E7F970136952795E7
:10597000892BA1F7C9018C0D9D1DB7010E94733AB7
:10598000FB01672B11F4E1E0F0E089819A8154E09A
:10599000880F991F5A95E1F7BF010E94733A9B0146
:1059A000C50144E0880F991F4A95E1F7BF010E94A5
:1059B000733A412F50E0153090F484E090E0841B5E
:1059C000950B082E02C0369527950A94E2F73A8384
:1059D000298302C0769567958A95E2F70FC0CA01C0
:1059E0000497082E02C0220F331F0A94E2F73A836D
:1059F000298302C0660F771F8A95E2F789819A8111
:105A0000892B21F481E090E09A83898361157105E7
:105A100011F461E070E0749718F4802F0E94580828
:105A200029814A8160E0892D0E94A005E02FF0E0E5
:105A3000E45CF94F81E0808322960FB6F894DEBFD4
:105A40000FBECDBFDF91CF911F910F91FF90EF90CF
:105A5000DF90CF90BF90AF909F9008950F931F93CA
:105A6000CF93DF93CDB7DEB762970FB6F894DEBF62
:105A70000FBECDBF082F162F8430C1F480E00E94E6
:105A8000412581E00E944125612F80E00E949326FC
:105A90006F83788789879A87612F81E00E94932698
:105AA0006B877C878D879E87198A3FC0853041F43C
:105AB00081E00E94412582E00E944125198625C08F
:105AC000863081F480E00E94412582E00E944125D9
:105AD000612F80E00E9493266F83788789879A8759
:105AE0001D861BC0873009F580E00E94412581E0BA
:105AF0000E94412582E00E944125612F80E00E94A2
:105B000093266F83788789879A87612F81E00E9427
:105B100093266B877C878D879E87612F82E00E940A
:105B200093266F87788B898B9A8B9985992331F48B
:105B30008D85882319F48989882369F09A83FE0169
:105B40003796818189838D858C838C858B83898928
:105B50008E8388890BC088858A838F8189838C8511
:105B60008C838B858B8388898E838F858D8304308E
:105B700049F429813A818B819C8182179307D0F463
:105B800041E015C0053049F42B813C818D819E8117
:105B90008217930758F041E00EC0063071F4298156
:105BA0003A818D819E818217930720F442E0BC01E7
:105BB000C90133C040E0B90130C0073081F58981A7
:105BC0009A812B813C81ED81FE812817390768F489
:105BD000E817F907C0F441E0B9010E94692C6D8112
:105BE0007E8142E089819A8118C0E217F30758F458
:105BF00040E0BC01C9010E94692C6D817E8142E0B8
:105C00008B819C810AC040E0BC01CF010E94692CBD
:105C10006B817C8141E08D819E810E94692C62961E
:105C20000FB6F894DEBF0FBECDBFDF91CF911F91AD
:105C30000F910895CF92DF92EF92FF920F931F93EF
:105C4000CF93DF93CDB7DEB724970FB6F894DEBFBE
:105C50000FBECDBF80913A06823008F04BC060E0A5
:105C600080913B060E94E40880913B060E944125FA
:105C70006E010894C11CD11C8091C5058C83809154
:105C8000C4058B838091C605F60181838091C80588
:105C9000898380913A06813009F5E980FA800B8189
:105CA0001C8180913B068295880F807E82600E94D5
:105CB0002908E60EF71E081F191FE982FA820B83D6
:105CC0001C838C818093C5058B818093C405F6016C
:105CD00081818093C60589818093C80549815A8155
:105CE0006B817C8180913B068295880F807E0E942B
:105CF000000946C0823009F043C0E090C805809199
:105D00003B06833030F40E9441256E2D80913B0686
:105D100035C06E2D0E942E2D80913B06843041F4BB
:105D20006E2D80E00E94C8266E2D81E00E94C8265C
:105D300080913B06853041F46E2D81E00E94C8269B
:105D40006E2D82E00E94C82680913B06863041F489
:105D50006E2D80E00E94C8266E2D82E00E94C8262B
:105D600080913B06873061F46E2D80E00E94C8264A
:105D70006E2D81E00E94C8266E2D82E00E94C8260A
:105D800024960FB6F894DEBF0FBECDBFDF91CF9142
:105D90001F910F91FF90EF90DF90CF900895CF92D9
:105DA000DF92EF92FF920F931F93CF93DF931092A6
:105DB0003806109237068FEF9FEF9093C7018093BC
:105DC000C6018DE090E00E94E60F813011F48093CF
:105DD000420618E4C12E16E0D12EBEE5EB2EB6E049
:105DE000FB2EC0E0D0E0CE018295880F807E182F78
:105DF0008C600E940F08F601819391936F01812FAF
:105E000086600E940F08F701819391937F0121968C
:105E1000C330D10541F70CEC14E0CEE1D3E0CE0164
:105E20000E94E60FF8018383CE0101970E94E60FDE
:105E3000F8018283CE0102970E94E60FF801818368
:105E4000CE0103970E94E60FF801808324960C5F31
:105E50001F4FF3E0CE3FDF0711F7ECEFFFE7E491D0
:105E6000E73299F4EDEFFFE7E491E83171F4EEEFFA
:105E7000FFE7E491E83249F4EFEFFFE7E491E8311E
:105E800021F481E08093EC0102C01092EC01DF91DB
:105E9000CF911F910F91FF90EF90DF90CF900895D9
:105EA0001F920F920FB60F9211248F939F93EF932F
:105EB000FF938BB1887129F08091ED01806280930E
:105EC000ED01869B04C08CB180931F021AC08091A3
:105ED00009029CB1E82FF0E0E251FE4F90838F5F02
:105EE000809309028B3110F01092090290910902FF
:105EF00080910A02981729F48091ED0180688093BF
:105F0000ED01FF91EF919F918F910F900FBE0F9038
:105F10001F9018951F920F920FB60F9211248F9316
:105F20009F93EF93FF9390911E0280911D0298170B
:105F300081F0969AE92FF0E0E55FFD4F80818CB902
:105F4000892F8F5F80931E02823120F010921E02F3
:105F500001C05598FF91EF919F918F910F900FBEC7
:105F60000F901F9018951F920F920FB60F92112449
:105F70008F939F9390911E0280911D02981709F4B0
:105F800096989F918F910F900FBE0F901F9018952C
:105F9000982F8091090280930A0280911E028093BB
:105FA0001D021092ED012091CD05283019F4EEE785
:105FB000F1E002C0E7E8F1E0849189B988ED8AB99F
:105FC000992369F0993058F4E92FF0E0283019F45A
:105FD000E258FE4F02C0E957FE4F849189B90895F7
:105FE0008091ED0181FF02C01092ED018BB18871AB
:105FF00029F08091ED0180628093ED018091ED01A7
:1060000082608093ED01807F19F08FEF9FEF0895FC
:1060100020E030E090910A0280910902981711F077
:1060200021E030E0C9010895969A90911D02E92F70
:10603000F0E0E55FFD4F80839F5F90931D029231FA
:1060400010F010921D0290911D0280911E0298176F
:1060500029F48091ED0180648093ED01559A0895B3
:10606000DC0190910A0280910902981719F480E0EE
:1060700090E00895E92FF0E0E251FE4F80818C938B
:10608000892F8F5F80930A028B3118F481E090E0B2
:10609000089510920A0281E090E0089520911D0277
:1060A0002E5F30911E02223138F080E090E03323E1
:1060B00049F481E090E0089580E090E0231711F426
:1060C00081E090E0089520E030E090911E02809100
:1060D0001D02981711F421E030E0C9010895EF92F4
:1060E000FF920F931F93CF93DF93CDB7DEB7229725
:1060F0000FB6F894DEBF0FBECDBF1A8219827E01A3
:106100000894E11CF11C46C08BB78F7B8BBFC498F1
:1061100086E00E949010C49A8BB780648BBF8BB7C7
:106120008F7B8BBFC49882E00E949010F701818121
:106130000E94901089810E94901000E010E08981F7
:106140009A81800F911F885F9F4340F480E00E94F6
:1061500090100F5F1F4F0034110589F7C49A8BB759
:1061600080648BBF00E010E01CC0C49A8BB78064D1
:106170008BBF0AC0C49A8BB780648BBF0F5F1F4F61
:106180002EE2003E120769F489819A81805C9F4F5C
:106190009A83898389819A818050904408F4B4CF8E
:1061A0000DC08BB78F7B8BBFC49885E00E94901089
:1061B00080E00E94901080FDDDCFD7CF22960FB6F1
:1061C000F894DEBF0FBECDBFDF91CF911F910F912D
:1061D000FF90EF900895EF92FF920F931F93CF934C
:1061E000DF937B018C0193E0000F111F9A95E1F77B
:1061F0008BB78F7B8BBFC49883E00E949010812F58
:1062000099270E949010802F0E949010C0E0D0E04B
:1062100087010C0F1D1F80E00E949010F801808301
:106220002196C830D105A1F7C49A8BB780648BBF83
:1062300080E090E0DF91CF911F910F91FF90EF9060
:106240000895EF92FF920F931F93CF93DF937B01FB
:106250008C0133E0000F111F3A95E1F78BB78F7B6C
:106260008BBFC49886E00E949010C49A8BB780645C
:106270008BBF8BB78F7B8BBFC49882E00E9490103E
:10628000812F99270E949010802F0E949010C0E0CB
:10629000D0E0F701EC0FFD1F80810E949010219645
:1062A000C830D105B1F7C49A8BB780648BBFC0E00A
:1062B000D0E013C0C49A8BB780648BBF80E090E0BD
:1062C00019C0C49A8BB780648BBF21968EE2C03E02
:1062D000D80719F48FEF9FEF0DC08BB78F7B8BBF63
:1062E000C49885E00E94901080E00E94901080FD8C
:1062F000E8CFE0CFDF91CF911F910F91FF90EF900A
:1063000008959091E40596959093E4058091E305B6
:1063100080FF03C090689093E4059091E305969503
:106320009093E3058091E20580FF03C0906890930D
:10633000E3058091E20586958093E20586FF03C020
:1063400080688093E2050895E82FF0E0EE0FFF1FCC
:10635000EF5CFD4F80819181009719F00197918347
:1063600080830895BF92CF92DF92EF92FF920F93B6
:106370001F93CF93DF93082FC82EDD24F601E05141
:10638000FA4F108123E0B22EB80E8B2D0E946D10B3
:10639000E601CC0FDD1F843098F48DE70E940208DF
:1063A00022E030E00C2E02C0220F331F0A94E2F7E5
:1063B000F82EF2228DE70E94020821E030E012C0A0
:1063C0008DE70E94020821E030E00C2E02C0220F6F
:1063D000331F0A94E2F7F82EF2228DE70E9402089A
:1063E00022E030E002C0220F331FCA95E2F7822379
:1063F000E02EE294EE0CB0EEEB22113019F5F6012E
:10640000EE0FFF1FEF5CFD4F1182108285E1E82A3D
:10641000E092D80561EE75E088ED95E00E94BC043D
:10642000F601E25DFD4F8091E305808362E0802FFD
:106430000E94E4088B2D0E946D10823008F4B8C1D0
:1064400012E0B7C1123051F4802F8A5F0E946D10A4
:10645000682F802F0E945E0913E0ABC1133021F436
:10646000882309F0A5C1A5C1143051F4802F8A5F9B
:106470000E946D10682F802F0E94410915E099C17C
:10648000153089F4FF2009F494C1802F0E94360949
:10649000F601EE0FFF1FEF5CFD4F8EE190E0918360
:1064A000808316E086C11630A1F4F601EE0FFF1FBF
:1064B000EF5CFD4F80819181892B09F07AC1802F9B
:1064C000875F0E946D10682F802F0E945E0917E081
:1064D00070C11730D9F4FF2009F06BC122E043E00E
:1064E00060E08E2D84610E94A00520E040E060E025
:1064F0008E2D8C610E94A005802F875F0E946D10F9
:10650000682F802F0E94410918E053C1183011F5FF
:10651000FF2009F44EC1802F0E9436098E2D8D6117
:106520008093D80561EE75E088ED95E00E94BC048B
:106530002091E4054091E3056091E2058E2D0E94D3
:10654000A00520E043E060E08E2D84610E94A0055C
:1065500019E02FC1193009F041C08DE78093D805AB
:1065600061EE75E088ED95E00E94BC048091E10544
:1065700090E09601220F331F02C0959587952A95CA
:10658000E2F780FF16C18B2D0E946D10182F62E07C
:10659000802F0E94E408802F0E94360920E040E00E
:1065A00060E08E2D0E94A00520E040E060E08E2D8E
:1065B00082600E94A005133039F0809120029091F2
:1065C0002102892B09F473C0802F875F0E946D1010
:1065D000682F802F0E9441091AE0EBC01A3061F445
:1065E000FF2009F4E6C020E040E060E08E2D8C61E1
:1065F0000E94A0051BE0DDC01B3009F05AC0FF203F
:1066000009F0D7C0802F0E9436098E2D8D618093AE
:10661000D80561EE75E088ED95E00E94BC040E940B
:1066200081312091E4054091E3056091E2058E2DD2
:106630000E94A00520E043E060E08E2D84610E946E
:10664000A0051091E40510951093E4050091E30571
:1066500000950093E305F090E205F094F092E205D6
:106660000E9481318091E405810F8093E4058823A5
:1066700029F48091E3058F5F8093E3058091E30522
:10668000800F8093E305882329F48091E2058F5FD2
:106690008093E2056091E2056F0D6093E205209121
:1066A000E4054091E3058E2D8A610E94A0051EE05D
:1066B00080C01E3009F06EC08091E10590E0960127
:1066C000220F331F02C0959587952A95E2F780FF28
:1066D00070C062E0802F0E94E408802F0E9436097B
:1066E0008B2D0E946D10833031F0809120029091AB
:1066F0002102892B91F01092E1051092E20510928F
:10670000E305F601EE0FFF1FEE0FFF1FEE5DFD4FDD
:10671000108211821282138203C08E2D0E941D0BE3
:106720002091E4054091E3056091E2058E2D0E94E1
:10673000A0051E2D12602091E4054091E3056091B3
:10674000E205812F0E94A00520E040E060E08E2D50
:106750000E94A00520E040E060E0812F0E94A0059B
:10676000F601E25DFD4F20E0408160E08E2D846106
:106770000E94A005F601EE0FFF1FE25AF94F40817B
:106780005181662757FD6095762F8E2D86600E9479
:1067900000090CC01F3069F4F601E25DFD4F22E0F4
:1067A000408160E08E2D84610E94A00510E001C050
:1067B00014E0E0EFF5E0CE0EDF1EF6011083DF916E
:1067C000CF911F910F91FF90EF90DF90CF90BF90EE
:1067D0000895AC018091A704882319F480E090E02B
:1067E00008958BB78F7B8BBF9091380280913702D1
:1067F000981711F490E01EC020913802822F90E08B
:10680000FC0134E0EE0FFF1F3A95E1F7E81BF90BAE
:10681000DA01E959FC4F8FE001900D928150E1F7C8
:106820002F5F2093380280913802843111F4109246
:10683000380291E08BB780648BBF892F90E0089578
:106840000F931F93CF93DF93DA9895E0909393047F
:10685000809394046093950440939604C0E0D0E044
:106860008E010D561B4FF80180810E949010F80197
:1068700080832196C430D10599F7DA9ADF91CF91C0
:106880001F910F910895EF92FF920F931F93CF9353
:10689000DF93DA9892E09093930480939404EE242B
:1068A000FF24C62FD0E0229609C08C010D561B4F45
:1068B000F80180810E949010F80180838E2D90E075
:1068C0000894E11CF11C8C179D077CF3DA9ADF9188
:1068D000CF911F910F91FF90EF9008950F931F9309
:1068E000CF93DF93DA9892E090939304809394048B
:1068F00060939504C0E0D0E08E010D561B4FF80167
:1069000080810E949010F80180832196C330D105C8
:1069100099F7DA9ADF91CF911F910F910895EF9235
:10692000FF920F931F93CF93DF93DA9893E09093A6
:10693000930480939404EE24FF24C62FD0E0229683
:1069400009C08C010D561B4FF80180810E949010E8
:10695000F80180838E2D90E00894E11CF11C8C17C7
:106960009D077CF3DA9ADF91CF911F910F91FF90F1
:10697000EF9008958F929F92AF92BF92CF92DF9245
:10698000EF92FF920F931F93CF93DF93EC014A0195
:106990005B016801790110923A0280913A0280937A
:1069A00039028091390280933802809138028093B5
:1069B000370264E88FE00E946E3461E08EE00E944E
:1069C0008F34809195048F3F19F41092A704CAC0A8
:1069D0008091950487FFF1CF81E08093A704C130B7
:1069E000D10511F467E211C0C230D10551F46FE056
:1069F0008AE20E946E346FEB89E20E946E3467E097
:106A000038C0C330D10531F467E08AE20E946E34A9
:106A10006AEBF2CFC430D10511F463E0F6CFC53094
:106A2000D10511F463E011C0C630D10551F463E023
:106A30008AE20E946E3468E989E20E946E3461E065
:106A400018C0C730D10551F460E08AE20E946E346C
:106A500068EB89E20E946E3465E00BC0289761F410
:106A600060E08AE20E946E3460E989E20E946E343E
:106A700062E088E20E946E3460E08DE00E946E3435
:106A800060E08CE00E946E34D501C40153E0B695FD
:106A9000A795979587955A95D1F780939504882D5A
:106AA0008295880F807E80939604109297041092AE
:106AB000980464E080E00E9443340FEF0093950453
:106AC00010EE10939604109297041092980464E0CC
:106AD00080E20E944334D701C60143E0B695A795F2
:106AE000979587954A95D1F7809395048C2D82953B
:106AF000880F807E809396041092970410929804D9
:106B000064E084E00E94433400939504109396045B
:106B1000109297041092980464E084E20E94433437
:106B200060E080E60E946E3460E080E70E946E3490
:106B3000C114D104E104F10411F063E101C061E189
:106B40008BE20E946E3464E08FE00E946E3461E05C
:106B50008EE00E948F348091950487FDF8CF8BB72B
:106B600080648BBFDF91CF911F910F91FF90EF90C9
:106B7000DF90CF90BF90AF909F908F900895AF928D
:106B8000BF92CF92DF92EF92FF920F931F9380916B
:106B9000340680FF0FC08091D4059091D505892BD4
:106BA00049F08091D4059091D50501979093D50532
:106BB0008093D4058091D6059091D705892BA9F1B2
:106BC0008091D4059091D505892B79F5DB9880E0EB
:106BD00000008F5F8436E1F7DB9A80E000008F5F72
:106BE0008436E1F7E090DC05F090DD050091DE05EC
:106BF0001091DF05A0903006B0903106C0903206AB
:106C0000D090330685E090E00E94E60F980187015E
:106C1000B601A50190E00E94BA348091D60590910A
:106C2000D7059093D5058093D4051F910F91FF90C0
:106C3000EF90DF90CF90BF90AF900895CF93DF9308
:106C4000EC01662319F46EE080E602C06EE080E796
:106C50000E948F34809197048695869586958170E1
:106C600089838981882309F458C080919A04829588
:106C70008695869581708A838091970490E0A0E044
:106C8000B0E0FBE1880F991FAA1FBB1FFA95D1F74F
:106C90008B839C83AD83BE832B813C814D815E8140
:106CA0008091980490E0A0E0B0E0E3E1880F991FA4
:106CB000AA1FBB1FEA95D1F7822B932BA42BB52BD0
:106CC0008B839C83AD83BE832B813C814D815E8110
:106CD0008091990490E0A0E0B0E07BE0880F991FDC
:106CE000AA1FBB1F7A95D1F7822B932BA42BB52B10
:106CF0008B839C83AD83BE832B813C814D815E81E0
:106D00008091970482958695877090E0A0E0B0E02E
:106D1000822B932BA42BB52B0FC0809195048695C5
:106D20008695869581708A83809197048295869551
:106D3000877090E0A0E0B0E08B839C83AD83BE833E
:106D40002B813C814D815E818091960490E063E0CF
:106D5000880F991F6A95E1F7AA2797FDA095BA2F8A
:106D6000822B932BA42BB52B8B839C83AD83BE836B
:106D700080919A048F70888320E030E0F901E55615
:106D8000FB4F8081F901EC0FFD1F87832F5F3F4F81
:106D90002830310599F7DF91CF910895AC018091AA
:106DA000A704882319F480E090E008958BB78F7BC7
:106DB0008BBF209139022F5F243109F420E08091AC
:106DC0003A02281711F490E023C08091390290E034
:106DD000FC01A4E0EE0FFF1FAA95E1F7E81BF90BF9
:106DE000E55CFD4FDA018FE00D9001928150E1F7F3
:106DF0002093390261E080E50E948F3480919504F0
:106E000083FD05C040E160E18CE20E94203491E006
:106E10008BB780648BBF892F90E008951F920F92EB
:106E20000FB60F9211241F932F933F934F935F93AD
:106E30006F937F938F939F93AF93BF93CF93DF9382
:106E4000EF93FF9361E08CE20E948F348091950470
:106E5000C82F80FF1CC0109137021F5F143109F446
:106E600010E080913802181769F0809137022FE006
:106E7000829FC001112460E089599C4F0E941E36F8
:106E80001093370240E061E08CE20E942034C1FFA1
:106E90001CC0109137021F5F143109F410E080917B
:106EA0003802181769F0809137022FE0829FC001E5
:106EB000112461E089599C4F0E941E3610933702BD
:106EC00040E062E08CE20E942034C4FF95C040E0C4
:106ED00060E18CE20E94203490913A028091390264
:106EE000981709F489C080913A029FE0899FE001D8
:106EF0001124C55CDD4F8F5F80933A028B819C81AA
:106F0000AD81BE81689412F8B695A795979587953F
:106F10001694D1F7809395048B819C81AD81BE81BD
:106F20008295880F807E8093960489818823B9F1A9
:106F300080919604886080939604209196048B81BA
:106F40009C81AD81BE814BE1B695A79597958795BC
:106F50004A95D1F78370822B8093960420919704F1
:106F60008B819C81AD81BE8133E1B695A7959795C4
:106F700087953A95D1F7282B209397042091980470
:106F80008B819C81AD81BE811BE0B695A7959795BD
:106F900087951A95D1F7282B2093980404C0109256
:106FA00097041092980488818F70809399048A8145
:106FB000882329F08091990480648093990420E0CB
:106FC00030E0F901EC0FFD1F8781F901E656FB4F18
:106FD00080832F5F3F4F2830310599F76DE081E5C1
:106FE0000E9443346BE080E50E946E3480913A0247
:106FF000843111F410923A02FF91EF91DF91CF9119
:10700000BF91AF919F918F917F916F915F914F91C0
:107010003F912F911F910F900FBE0F901F901895C9
:10702000823010F482E001C08E7F82B985EC86BF89
:1070300085B3836085BB0895DC019091A804961701
:1070400019F080E090E0089540E020E030E00BC0CF
:10705000F901E555FB4F8081FD01E20FF31F8083AD
:107060004F5F2F5F3F4F491799F71092A80481E0B7
:1070700090E00895DC0140E020E030E00BC0FD012D
:10708000E20FF31F8081F901EC54FB4F80834F5FC7
:107090002F5F3F4F461799F76093AA0408951F92F8
:1070A0000F920FB60F9211248F939F93EF93FF933C
:1070B00081B1803629F485EC86BF1092A80453C0B4
:1070C00081B1803819F081B1883871F485EC86BFC0
:1070D0008091A804E82FF0E093B1E555FB4F908331
:1070E0008F5F8093A8043FC081B1803AD1F181B114
:1070F000882311F485ED36C081B1883AB1F410923D
:10710000A9049091A904E92FF0E0EC54FB4F808191
:1071100083B99F5F9093A90485EC86BF9091A904E1
:107120008091AA049817F9F416C081B1883BC9F47C
:107130009091A904E92FF0E0EC54FB4F808183B9D2
:107140009F5F9093A90485EC86BF9091A9048091DC
:10715000AA04981741F48091A90481508093A9044E
:1071600002C085EC86BFFF91EF919F918F910F90A8
:107170000FBE0F901F901895FF920F931F93982F9B
:10718000162F042FF22E8091BD04813029F48BB785
:107190008F7B8BBFAF980DC0823029F48BB78F7B6C
:1071A0008BBFAE9806C0833021F48BB78F7B8BBF2B
:1071B000AD98892F0E949010812F0E949010802FEF
:1071C0000E9490108F2D0E94901085B3806E85BB19
:1071D0008BB780648BBF1F910F91FF900895CF9361
:1071E000DF93CDB7DEB724970FB6F894DEBF0FBE9E
:1071F000CDBF49835A836B837C83813011F48AE04D
:1072000005C0823011F48CE001C088E029814A81F8
:107210006B8181600E94BC3824960FB6F894DEBF63
:107220000FBECDBFDF91CF910895CF93DF93CDB740
:10723000DEB724970FB6F894DEBF0FBECDBF88230C
:1072400011F4E0E005C0813011F4E2E001C0E4E0B7
:10725000842F90E09695982F882797958795A0E0A2
:10726000B0E09B0140E050E06CE0220F331F441F70
:10727000551F6A95D1F7822B932BA42BB52B8983AD
:107280009A83AB83BC8329814A816B818E2F816075
:107290000E94BC3824960FB6F894DEBF0FBECDBF57
:1072A000DF91CF91089520E040E064E087E00E9404
:1072B000BC3820E040E060E281E10E94BC3820E080
:1072C00040E060E089E00E94BC3820E040E060E0FF
:1072D0008BE00E94BC3820E040E060E08DE00E943E
:1072E000BC380895CF92DF92EF92FF920F931F93D5
:1072F000CF93DF936C017B018091BD04813029F431
:107300008BB78F7B8BBFAF980DC0823029F48BB7C2
:107310008F7B8BBFAE9806C0833021F48BB78F7BF9
:107320008BBFAD98C0E0D0E087010C0F1D1FF601A8
:10733000EC0FFD1F80810E949010F8018083219640
:10734000C430D10589F785B3806E85BB8BB7806467
:107350008BBFDF91CF911F910F91FF90EF90DF9046
:10736000CF900895CF93DF93CDB7DEB72C970FB6AC
:10737000F894DEBF0FBECDBF813011F48AE005C0A6
:10738000823011F48CE001C088E08D83BE016F5F14
:107390007F4FCE0105960E9472391C868A818B87A9
:1073A0009B819A879C81998787FF03C08FEF8C8789
:1073B00001C01C8669857A858B859C852C960FB6C5
:1073C000F894DEBF0FBECDBFDF91CF910895A0E04E
:1073D000B0E0EDEEF9E30C94F33AEC0168817981C9
:1073E0008A819B81611571058105910549F484E2CB
:1073F000A82E89EDB82E8BE5C82E87E0D82E02C0C6
:107400005B016C01C601B5012DE133EF41E050E0B5
:107410000E949A3A27EA31E440E050E00E94543A50
:107420007B018C01C601B5012DE133EF41E050E055
:107430000E949A3ACA01B90124E13BE040E050E0E1
:107440000E94543AE61AF70A080B190B17FF08C0F6
:107450008FEF9FEFAFEFBFE7E80EF91E0A1F1B1F6C
:10746000E882F9820A831B838FEF9FEFAFEFBFE7BC
:10747000E822F9220A231B23C801B701EAE0CDB7AD
:10748000DEB70C940F3B0E94E73908958CE091E041
:107490000E94E739089560930C0170930D01809369
:1074A0000E0190930F010895629FD001739FF00128
:1074B000829FE00DF11D649FE00DF11D929FF00D84
:1074C000839FF00D749FF00D659FF00D9927729FBB
:1074D000B00DE11DF91F639FB00DE11DF91FBD0146
:1074E000CF0111240895AA1BBB1B51E107C0AA1F9D
:1074F000BB1FA617B70710F0A61BB70B881F991F55
:107500005A95A9F780959095BC01CD01089597FBF8
:10751000092E07260AD077FD04D0E5DF06D000202B
:107520001AF4709561957F4F0895F6F790958195BF
:107530009F4F089597FB092E05260ED057FD04D0C6
:1075400014D00AD0001C38F4509540953095219500
:107550003F4F4F4F5F4F0895F6F790958095709588
:1075600061957F4F8F4F9F4F0895A1E21A2EAA1B5E
:10757000BB1BFD010DC0AA1FBB1FEE1FFF1FA217E3
:10758000B307E407F50720F0A21BB30BE40BF50BE0
:10759000661F771F881F991F1A9469F76095709569
:1075A000809590959B01AC01BD01CF010895E199B3
:1075B000FECFBFBBAEBBE09A11960DB20895E19924
:1075C000FECFBFBBAEBB0DBA11960FB6F894E29AD0
:1075D000E19A0FBE08952F923F924F925F926F9261
:1075E0007F928F929F92AF92BF92CF92DF92EF9253
:1075F000FF920F931F93CF93DF93CDB7DEB7CA1BD4
:10760000DB0B0FB6F894DEBF0FBECDBF09942A88FE
:10761000398848885F846E847D848C849B84AA84A6
:10762000B984C884DF80EE80FD800C811B81AA8133
:10763000B981CE0FD11D0FB6F894DEBF0FBECDBFFE
:06764000ED010895FFCFEB
:10764600A911C0257625181B1A2EDE2616235522CB
:107656008C213C1F5E1D391C221BCE1A5129D528B0
:10766600AB11AD11AF11B111D6131D14A214AB1489
:10767600C714DA14E114A219E814DE187B181F18CF
:107686005626AE12B6286D21EB1426153315341581
:10769600361538153A153C153E1540154215441554
:1076A600461548154A154C154E15501552155415C4
:1076B600561558155A155C155E1560156215641534
:1076C60003040A0404040504060407040804090460
:1076D6006615691579157D15A917A2157E17A915C1
:1076E60055176B18F9150F16BB1613160100000077
:00000001FF
